 objfree002

 Timestamp is c9a652cb (reproducible build file hash)

 Preferred load address is 0000000180000000

 Start         Length     Name                   Class
 0001:00000000 00003b80H .text$mn                CODE
 0001:00003b80 00000036H .text$mn$00             CODE
 0001:00003bb6 00000092H .text$x                 CODE
 0002:00000000 000001c8H .idata$5                DATA
 0002:000001c8 00000038H .00cfg                  DATA
 0002:00000200 00000008H .CRT$XCA                DATA
 0002:00000208 00000008H .CRT$XCZ                DATA
 0002:00000210 00000008H .CRT$XIA                DATA
 0002:00000218 00000008H .CRT$XIC                DATA
 0002:00000220 00000008H .CRT$XIZ                DATA
 0002:00000228 00000008H .CRT$XLA                DATA
 0002:00000230 00000008H .CRT$XLZ                DATA
 0002:00000238 00000008H .CRT$XPA                DATA
 0002:00000240 00000008H .CRT$XPZ                DATA
 0002:00000248 00000008H .CRT$XTA                DATA
 0002:00000250 00000010H .CRT$XTZ                DATA
 0002:00000258 00000000H .gehcont$y              DATA
 0002:00000258 00000000H .gfids$y                DATA
 0002:00000260 000029a0H .rdata                  DATA
 0002:00002c00 00000000H .rdata$CastGuardVftablesA DATA
 0002:00002c00 00000000H .rdata$CastGuardVftablesC DATA
 0002:00002c00 00000028H .rdata$T                DATA
 0002:00002c28 000000fcH .rdata$voltmd           DATA
 0002:00002d24 0000031cH .rdata$zzzdbg           DATA
 0002:00003040 00000008H .rtc$IAA                DATA
 0002:00003048 00000008H .rtc$IZZ                DATA
 0002:00003050 00000008H .rtc$TAA                DATA
 0002:00003058 00000008H .rtc$TZZ                DATA
 0002:00003060 00000004H .tls                    DATA
 0002:00003064 00000004H .tls$                   DATA
 0002:00003068 00000008H .tls$ZZZ                DATA
 0002:00003070 00000360H .xdata                  DATA
 0002:000033d0 000003d0H .edata                  DATA
 0002:000037a0 0000008cH .idata$2                DATA
 0002:0000382c 00000014H .idata$3                DATA
 0002:00003840 000001c8H .idata$4                DATA
 0002:00003a08 00000486H .idata$6                DATA
 0003:00000000 00000080H .data                   DATA
 0003:00000080 0001b798H .bss                    DATA
 0004:00000000 000003ccH .pdata                  DATA

  Address         Publics by Value              Rva+Base               Lib:Object

 0000:00000000       __AbsoluteZero             0000000000000000     <absolute>
 0000:00000000       ___safe_se_handler_count   0000000000000000     <absolute>
 0000:00000000       ___safe_se_handler_table   0000000000000000     <absolute>
 0000:00000000       __arm64x_extra_rfe_table   0000000000000000     <absolute>
 0000:00000000       __arm64x_extra_rfe_table_size 0000000000000000     <absolute>
 0000:00000000       __arm64x_native_entrypoint 0000000000000000     <absolute>
 0000:00000000       __arm64x_redirection_metadata 0000000000000000     <absolute>
 0000:00000000       __arm64x_redirection_metadata_count 0000000000000000     <absolute>
 0000:00000000       __dynamic_value_reloc_table 0000000000000000     <absolute>
 0000:00000000       __enclave_config           0000000000000000     <absolute>
 0000:00000000       __guard_check_icall_a64n_fptr 0000000000000000     <absolute>
 0000:00000000       __guard_eh_cont_count      0000000000000000     <absolute>
 0000:00000000       __guard_eh_cont_table      0000000000000000     <absolute>
 0000:00000000       __guard_fids_count         0000000000000000     <absolute>
 0000:00000000       __guard_fids_table         0000000000000000     <absolute>
 0000:00000000       __guard_iat_count          0000000000000000     <absolute>
 0000:00000000       __guard_iat_table          0000000000000000     <absolute>
 0000:00000000       __guard_longjmp_count      0000000000000000     <absolute>
 0000:00000000       __guard_longjmp_table      0000000000000000     <absolute>
 0000:00000000       __hybrid_auxiliary_iat     0000000000000000     <absolute>
 0000:00000000       __hybrid_auxiliary_iat_copy 0000000000000000     <absolute>
 0000:00000000       __hybrid_code_map          0000000000000000     <absolute>
 0000:00000000       __hybrid_code_map_count    0000000000000000     <absolute>
 0000:00000000       __x64_code_ranges_to_entry_points 0000000000000000     <absolute>
 0000:00000000       __x64_code_ranges_to_entry_points_count 0000000000000000     <absolute>
 0000:00000100       __guard_flags              0000000000000100     <absolute>
 0000:00000000       __ImageBase                0000000180000000     <linker-defined>
 0001:00000000       ?NewObject@JNIEnv_@@QEAAPEAV_jobject@@PEAV_jclass@@PEAU_jmethodID@@ZZ 0000000180001000 f i libobjfree002.obj
 0001:00000024       ?SetEventNotificationMode@_jvmtiEnv@@QEAA?AW4jvmtiError@@W4jvmtiEventMode@@W4jvmtiEvent@@PEAV_jobject@@ZZ 0000000180001024 f i libobjfree002.obj
 0001:0000002c       ?TranslateError@@YAPEBDW4jvmtiError@@@Z 000000018000102c f   libobjfree002.obj
 0001:000002e4       ?nsk_jni_check_exception@@YAHPEAUJNIEnv_@@QEBDH@Z 00000001800012e4 f   libobjfree002.obj
 0001:00000428       ?nsk_jni_lverify@@YAHHPEAUJNIEnv_@@HQEBDH1ZZ 0000000180001428 f   libobjfree002.obj
 0001:000004c8       Agent_Initialize           00000001800014c8 f   libobjfree002.obj
 0001:00000854       Agent_OnAttach             0000000180001854 f   libobjfree002.obj
 0001:00000854       Agent_OnLoad               0000000180001854 f   libobjfree002.obj
 0001:0000085c       Java_nsk_jvmti_ObjectFree_objfree002_check 000000018000185c f   libobjfree002.obj
 0001:00000864       Java_nsk_jvmti_ObjectFree_objfree002_setTag 0000000180001864 f   libobjfree002.obj
 0001:00000964       Java_nsk_jvmti_unit_FollowReferences_FollowRefObjects_addRefToVerify 0000000180001964 f   libobjfree002.obj
 0001:00000b20       Java_nsk_jvmti_unit_FollowReferences_FollowRefObjects_getTag 0000000180001b20 f   libobjfree002.obj
 0001:00000bdc       Java_nsk_jvmti_unit_FollowReferences_FollowRefObjects_resetRefsToVerify 0000000180001bdc f   libobjfree002.obj
 0001:00000be4       Java_nsk_jvmti_unit_FollowReferences_FollowRefObjects_resetTags 0000000180001be4 f   libobjfree002.obj
 0001:00000c28       Java_nsk_jvmti_unit_FollowReferences_FollowRefObjects_setTag 0000000180001c28 f   libobjfree002.obj
 0001:00000e74       Java_nsk_share_jvmti_ArgumentHandler_getAgentOptionsString 0000000180001e74 f   libobjfree002.obj
 0001:00000f20       Java_nsk_share_jvmti_DebugeeClass_checkStatus 0000000180001f20 f   libobjfree002.obj
 0001:00000fa8       Java_nsk_share_jvmti_DebugeeClass_resetAgentData 0000000180001fa8 f   libobjfree002.obj
 0001:00001008       Java_nsk_share_jvmti_RedefineAgent_agentStatus 0000000180002008 f   libobjfree002.obj
 0001:00001014       Java_nsk_share_jvmti_RedefineAgent_isRedefined 0000000180002014 f   libobjfree002.obj
 0001:00001020       Java_nsk_share_jvmti_RedefineAgent_redefineAttempted 0000000180002020 f   libobjfree002.obj
 0001:0000102c       MA_checkStatus             000000018000202c f   libobjfree002.obj
 0001:000010d0       ObjectFree                 00000001800020d0 f   libobjfree002.obj
 0001:000012ec       VMDeath                    00000001800022ec f   libobjfree002.obj
 0001:00001344       __local_stdio_printf_options 0000000180002344 f i libobjfree002.obj
 0001:000018a4       exitOnError                00000001800028a4 f   libobjfree002.obj
 0001:00001958       fprintf                    0000000180002958 f i libobjfree002.obj
 0001:0000199c       nsk_complain               000000018000299c f   libobjfree002.obj
 0001:000019c8       nsk_jvmti_createJVMTIEnv   00000001800029c8 f   libobjfree002.obj
 0001:00001af8       nsk_jvmti_lverify          0000000180002af8 f   libobjfree002.obj
 0001:00001be8       nsk_jvmti_parseOptions     0000000180002be8 f   libobjfree002.obj
 0001:00001e38       nsk_jvmti_resetAgentData   0000000180002e38 f   libobjfree002.obj
 0001:00001eac       nsk_lcomplain              0000000180002eac f   libobjfree002.obj
 0001:00001ecc       nsk_ldisplay               0000000180002ecc f   libobjfree002.obj
 0001:00001eec       nsk_ltrace                 0000000180002eec f   libobjfree002.obj
 0001:00001f0c       nsk_lvcomplain             0000000180002f0c f   libobjfree002.obj
 0001:000020c4       nsk_lvdisplay              00000001800030c4 f   libobjfree002.obj
 0001:00002110       nsk_lverify                0000000180003110 f   libobjfree002.obj
 0001:0000216c       nsk_lvtrace                000000018000316c f   libobjfree002.obj
 0001:000021cc       nsk_printf                 00000001800031cc f   libobjfree002.obj
 0001:000021f4       nsk_vprintf                00000001800031f4 f   libobjfree002.obj
 0001:000022a8       printf                     00000001800032a8 f i libobjfree002.obj
 0001:00002c60       __raise_securityfailure    0000000180003c60 f   MSVCRT:gs_report.obj
 0001:00002c94       __report_gsfailure         0000000180003c94 f   MSVCRT:gs_report.obj
 0001:00002ed4       __GSHandlerCheck           0000000180003ed4 f   MSVCRT:gshandler.obj
 0001:00002ef4       __GSHandlerCheckCommon     0000000180003ef4 f   MSVCRT:gshandler.obj
 0001:00002f60       __security_check_cookie    0000000180003f60 f   MSVCRT:amdsecgs.obj
 0001:000032a0       _DllMainCRTStartup         00000001800042a0 f   MSVCRT:dll_dllmain.obj
 0001:000032e0       __scrt_acquire_startup_lock 00000001800042e0 f   MSVCRT:utility.obj
 0001:0000331c       __scrt_dllmain_after_initialize_c 000000018000431c f   MSVCRT:utility.obj
 0001:00003350       __scrt_dllmain_before_initialize_c 0000000180004350 f   MSVCRT:utility.obj
 0001:00003368       __scrt_dllmain_crt_thread_attach 0000000180004368 f   MSVCRT:utility.obj
 0001:00003390       __scrt_dllmain_crt_thread_detach 0000000180004390 f   MSVCRT:utility.obj
 0001:000033a8       __scrt_dllmain_exception_filter 00000001800043a8 f   MSVCRT:utility.obj
 0001:00003408       __scrt_dllmain_uninitialize_c 0000000180004408 f   MSVCRT:utility.obj
 0001:00003438       __scrt_dllmain_uninitialize_critical 0000000180004438 f   MSVCRT:utility.obj
 0001:0000344c       __scrt_initialize_crt      000000018000444c f   MSVCRT:utility.obj
 0001:00003498       __scrt_initialize_onexit_tables 0000000180004498 f   MSVCRT:utility.obj
 0001:00003524       __scrt_is_nonwritable_in_current_image 0000000180004524 f   MSVCRT:utility.obj
 0001:000035bc       __scrt_release_startup_lock 00000001800045bc f   MSVCRT:utility.obj
 0001:000035e0       __scrt_uninitialize_crt    00000001800045e0 f   MSVCRT:utility.obj
 0001:0000360c       _onexit                    000000018000460c f   MSVCRT:utility.obj
 0001:00003648       atexit                     0000000180004648 f   MSVCRT:utility.obj
 0001:00003660       __crt_debugger_hook        0000000180004660 f   MSVCRT:utility_desktop.obj
 0001:00003668       __scrt_fastfail            0000000180004668 f   MSVCRT:utility_desktop.obj
 0001:000037b4       _guard_check_icall_nop     00000001800047b4 f i MSVCRT:guard_support.obj
 0001:000037b8       __security_init_cookie     00000001800047b8 f   MSVCRT:gs_support.obj
 0001:00003864       DllMain                    0000000180004864 f   MSVCRT:dll_dllmain_stub.obj
 0001:00003888       ?__scrt_initialize_type_info@@YAXXZ 0000000180004888 f   MSVCRT:tncleanup.obj
 0001:00003898       ?__scrt_uninitialize_type_info@@YAXXZ 0000000180004898 f   MSVCRT:tncleanup.obj
 0001:000038a4       __local_stdio_scanf_options 00000001800048a4 f i MSVCRT:default_local_stdio_options.obj
 0001:000038ac       __scrt_initialize_default_local_stdio_options 00000001800048ac f   MSVCRT:default_local_stdio_options.obj
 0001:000038c8       __scrt_get_dyn_tls_init_callback 00000001800048c8 f   MSVCRT:dyn_tls_init.obj
 0001:000038d0       _RTC_Initialize            00000001800048d0 f   MSVCRT:initsect.obj
 0001:0000390c       _RTC_Terminate             000000018000490c f   MSVCRT:initsect.obj
 0001:00003948       __isa_available_init       0000000180004948 f   MSVCRT:cpu_disp.obj
 0001:00003af4       _get_startup_argv_mode     0000000180004af4 f   MSVCRT:argv_mode.obj
 0001:00003afc       __scrt_is_ucrt_dll_in_use  0000000180004afc f   MSVCRT:ucrt_detection.obj
 0001:00003b10       memcpy                     0000000180004b10 f   vcruntime:VCRUNTIME140.dll
 0001:00003b16       memset                     0000000180004b16 f   vcruntime:VCRUNTIME140.dll
 0001:00003b1c       strchr                     0000000180004b1c f   vcruntime:VCRUNTIME140.dll
 0001:00003b22       __C_specific_handler       0000000180004b22 f   vcruntime:VCRUNTIME140.dll
 0001:00003b28       __std_type_info_destroy_list 0000000180004b28 f   vcruntime:VCRUNTIME140.dll
 0001:00003b2e       strcmp                     0000000180004b2e f   ucrt:api-ms-win-crt-string-l1-1-0.dll
 0001:00003b34       strlen                     0000000180004b34 f   ucrt:api-ms-win-crt-string-l1-1-0.dll
 0001:00003b3a       _initterm                  0000000180004b3a f   ucrt:api-ms-win-crt-runtime-l1-1-0.dll
 0001:00003b40       _initterm_e                0000000180004b40 f   ucrt:api-ms-win-crt-runtime-l1-1-0.dll
 0001:00003b46       _seh_filter_dll            0000000180004b46 f   ucrt:api-ms-win-crt-runtime-l1-1-0.dll
 0001:00003b4c       _configure_narrow_argv     0000000180004b4c f   ucrt:api-ms-win-crt-runtime-l1-1-0.dll
 0001:00003b52       _initialize_narrow_environment 0000000180004b52 f   ucrt:api-ms-win-crt-runtime-l1-1-0.dll
 0001:00003b58       _initialize_onexit_table   0000000180004b58 f   ucrt:api-ms-win-crt-runtime-l1-1-0.dll
 0001:00003b5e       _register_onexit_function  0000000180004b5e f   ucrt:api-ms-win-crt-runtime-l1-1-0.dll
 0001:00003b64       _execute_onexit_table      0000000180004b64 f   ucrt:api-ms-win-crt-runtime-l1-1-0.dll
 0001:00003b6a       _crt_atexit                0000000180004b6a f   ucrt:api-ms-win-crt-runtime-l1-1-0.dll
 0001:00003b70       _cexit                     0000000180004b70 f   ucrt:api-ms-win-crt-runtime-l1-1-0.dll
 0001:00003b78       __acrt_initialize          0000000180004b78 f   MSVCRT:ucrt_stubs.obj
 0001:00003b78       __acrt_thread_attach       0000000180004b78 f   MSVCRT:ucrt_stubs.obj
 0001:00003b78       __acrt_thread_detach       0000000180004b78 f   MSVCRT:ucrt_stubs.obj
 0001:00003b78       __acrt_uninitialize        0000000180004b78 f   MSVCRT:ucrt_stubs.obj
 0001:00003b78       __acrt_uninitialize_critical 0000000180004b78 f   MSVCRT:ucrt_stubs.obj
 0001:00003b78       __scrt_stub_for_acrt_initialize 0000000180004b78 f   MSVCRT:ucrt_stubs.obj
 0001:00003b78       __scrt_stub_for_acrt_thread_attach 0000000180004b78 f   MSVCRT:ucrt_stubs.obj
 0001:00003b78       __scrt_stub_for_acrt_thread_detach 0000000180004b78 f   MSVCRT:ucrt_stubs.obj
 0001:00003b78       __scrt_stub_for_acrt_uninitialize 0000000180004b78 f   MSVCRT:ucrt_stubs.obj
 0001:00003b78       __scrt_stub_for_acrt_uninitialize_critical 0000000180004b78 f   MSVCRT:ucrt_stubs.obj
 0001:00003b78       __vcrt_initialize          0000000180004b78 f   MSVCRT:ucrt_stubs.obj
 0001:00003b78       __vcrt_thread_attach       0000000180004b78 f   MSVCRT:ucrt_stubs.obj
 0001:00003b78       __vcrt_thread_detach       0000000180004b78 f   MSVCRT:ucrt_stubs.obj
 0001:00003b78       __vcrt_uninitialize        0000000180004b78 f   MSVCRT:ucrt_stubs.obj
 0001:00003b78       __vcrt_uninitialize_critical 0000000180004b78 f   MSVCRT:ucrt_stubs.obj
 0001:00003b7c       __scrt_stub_for_is_c_termination_complete 0000000180004b7c f   MSVCRT:ucrt_stubs.obj
 0001:00003b7c       _is_c_termination_complete 0000000180004b7c f   MSVCRT:ucrt_stubs.obj
 0001:00003b90       _guard_dispatch_icall_nop  0000000180004b90 f   MSVCRT:guard_dispatch.obj
 0001:00003bb0       _guard_xfg_dispatch_icall_nop 0000000180004bb0 f   MSVCRT:guard_xfg_dispatch.obj
 0002:00000000       __imp_RtlCaptureContext    0000000180005000     kernel32:KERNEL32.dll
 0002:00000008       __imp_RtlLookupFunctionEntry 0000000180005008     kernel32:KERNEL32.dll
 0002:00000010       __imp_RtlVirtualUnwind     0000000180005010     kernel32:KERNEL32.dll
 0002:00000018       __imp_UnhandledExceptionFilter 0000000180005018     kernel32:KERNEL32.dll
 0002:00000020       __imp_SetUnhandledExceptionFilter 0000000180005020     kernel32:KERNEL32.dll
 0002:00000028       __imp_GetCurrentProcess    0000000180005028     kernel32:KERNEL32.dll
 0002:00000030       __imp_TerminateProcess     0000000180005030     kernel32:KERNEL32.dll
 0002:00000038       __imp_IsProcessorFeaturePresent 0000000180005038     kernel32:KERNEL32.dll
 0002:00000040       __imp_CloseHandle          0000000180005040     kernel32:KERNEL32.dll
 0002:00000048       __imp_InitializeCriticalSectionAndSpinCount 0000000180005048     kernel32:KERNEL32.dll
 0002:00000050       __imp_DeleteCriticalSection 0000000180005050     kernel32:KERNEL32.dll
 0002:00000058       __imp_CreateEventW         0000000180005058     kernel32:KERNEL32.dll
 0002:00000060       __imp_GetModuleHandleW     0000000180005060     kernel32:KERNEL32.dll
 0002:00000068       __imp_GetProcAddress       0000000180005068     kernel32:KERNEL32.dll
 0002:00000070       __imp_IsDebuggerPresent    0000000180005070     kernel32:KERNEL32.dll
 0002:00000078       __imp_QueryPerformanceCounter 0000000180005078     kernel32:KERNEL32.dll
 0002:00000080       __imp_GetCurrentProcessId  0000000180005080     kernel32:KERNEL32.dll
 0002:00000088       __imp_GetCurrentThreadId   0000000180005088     kernel32:KERNEL32.dll
 0002:00000090       __imp_GetSystemTimeAsFileTime 0000000180005090     kernel32:KERNEL32.dll
 0002:00000098       __imp_DisableThreadLibraryCalls 0000000180005098     kernel32:KERNEL32.dll
 0002:000000a0       __imp_InitializeSListHead  00000001800050a0     kernel32:KERNEL32.dll
 0002:000000a8       \177KERNEL32_NULL_THUNK_DATA 00000001800050a8     kernel32:KERNEL32.dll
 0002:000000b0       __imp_memcpy               00000001800050b0     vcruntime:VCRUNTIME140.dll
 0002:000000b8       __imp_memset               00000001800050b8     vcruntime:VCRUNTIME140.dll
 0002:000000c0       __imp_strchr               00000001800050c0     vcruntime:VCRUNTIME140.dll
 0002:000000c8       __imp___C_specific_handler 00000001800050c8     vcruntime:VCRUNTIME140.dll
 0002:000000d0       __imp___std_type_info_destroy_list 00000001800050d0     vcruntime:VCRUNTIME140.dll
 0002:000000d8       \177VCRUNTIME140_NULL_THUNK_DATA 00000001800050d8     vcruntime:VCRUNTIME140.dll
 0002:000000e0       __imp_strtol               00000001800050e0     ucrt:api-ms-win-crt-convert-l1-1-0.dll
 0002:000000e8       \177api-ms-win-crt-convert-l1-1-0_NULL_THUNK_DATA 00000001800050e8     ucrt:api-ms-win-crt-convert-l1-1-0.dll
 0002:000000f0       __imp_malloc               00000001800050f0     ucrt:api-ms-win-crt-heap-l1-1-0.dll
 0002:000000f8       __imp_free                 00000001800050f8     ucrt:api-ms-win-crt-heap-l1-1-0.dll
 0002:00000100       \177api-ms-win-crt-heap-l1-1-0_NULL_THUNK_DATA 0000000180005100     ucrt:api-ms-win-crt-heap-l1-1-0.dll
 0002:00000108       __imp__errno               0000000180005108     ucrt:api-ms-win-crt-runtime-l1-1-0.dll
 0002:00000110       __imp_exit                 0000000180005110     ucrt:api-ms-win-crt-runtime-l1-1-0.dll
 0002:00000118       __imp__cexit               0000000180005118     ucrt:api-ms-win-crt-runtime-l1-1-0.dll
 0002:00000120       __imp__crt_atexit          0000000180005120     ucrt:api-ms-win-crt-runtime-l1-1-0.dll
 0002:00000128       __imp__execute_onexit_table 0000000180005128     ucrt:api-ms-win-crt-runtime-l1-1-0.dll
 0002:00000130       __imp__register_onexit_function 0000000180005130     ucrt:api-ms-win-crt-runtime-l1-1-0.dll
 0002:00000138       __imp__initialize_onexit_table 0000000180005138     ucrt:api-ms-win-crt-runtime-l1-1-0.dll
 0002:00000140       __imp__initialize_narrow_environment 0000000180005140     ucrt:api-ms-win-crt-runtime-l1-1-0.dll
 0002:00000148       __imp__configure_narrow_argv 0000000180005148     ucrt:api-ms-win-crt-runtime-l1-1-0.dll
 0002:00000150       __imp__seh_filter_dll      0000000180005150     ucrt:api-ms-win-crt-runtime-l1-1-0.dll
 0002:00000158       __imp__initterm_e          0000000180005158     ucrt:api-ms-win-crt-runtime-l1-1-0.dll
 0002:00000160       __imp__initterm            0000000180005160     ucrt:api-ms-win-crt-runtime-l1-1-0.dll
 0002:00000168       \177api-ms-win-crt-runtime-l1-1-0_NULL_THUNK_DATA 0000000180005168     ucrt:api-ms-win-crt-runtime-l1-1-0.dll
 0002:00000170       __imp___acrt_iob_func      0000000180005170     ucrt:api-ms-win-crt-stdio-l1-1-0.dll
 0002:00000178       __imp_fflush               0000000180005178     ucrt:api-ms-win-crt-stdio-l1-1-0.dll
 0002:00000180       __imp___stdio_common_vsprintf 0000000180005180     ucrt:api-ms-win-crt-stdio-l1-1-0.dll
 0002:00000188       __imp___stdio_common_vfprintf 0000000180005188     ucrt:api-ms-win-crt-stdio-l1-1-0.dll
 0002:00000190       \177api-ms-win-crt-stdio-l1-1-0_NULL_THUNK_DATA 0000000180005190     ucrt:api-ms-win-crt-stdio-l1-1-0.dll
 0002:00000198       __imp_strcmp               0000000180005198     ucrt:api-ms-win-crt-string-l1-1-0.dll
 0002:000001a0       __imp__strdup              00000001800051a0     ucrt:api-ms-win-crt-string-l1-1-0.dll
 0002:000001a0       __imp_strdup               00000001800051a0     ucrt:api-ms-win-crt-string-l1-1-0.dll
 0002:000001a8       __imp_strlen               00000001800051a8     ucrt:api-ms-win-crt-string-l1-1-0.dll
 0002:000001b0       __imp_strpbrk              00000001800051b0     ucrt:api-ms-win-crt-string-l1-1-0.dll
 0002:000001b8       __imp_strncpy              00000001800051b8     ucrt:api-ms-win-crt-string-l1-1-0.dll
 0002:000001c0       \177api-ms-win-crt-string-l1-1-0_NULL_THUNK_DATA 00000001800051c0     ucrt:api-ms-win-crt-string-l1-1-0.dll
 0002:000001c8       __guard_check_icall_fptr   00000001800051c8     MSVCRT:guard_support.obj
 0002:000001d0       __guard_xfg_check_icall_fptr 00000001800051d0     MSVCRT:guard_support.obj
 0002:000001d8       __guard_dispatch_icall_fptr 00000001800051d8     MSVCRT:guard_support.obj
 0002:000001e0       __guard_xfg_dispatch_icall_fptr 00000001800051e0     MSVCRT:guard_support.obj
 0002:000001e8       __guard_xfg_table_dispatch_icall_fptr 00000001800051e8     MSVCRT:guard_support.obj
 0002:000001f0       __castguard_check_failure_os_handled_fptr 00000001800051f0     MSVCRT:guard_support.obj
 0002:000001f8       __guard_memcpy_fptr        00000001800051f8     vcruntime:softmemtag.obj
 0002:00000200       __xc_a                     0000000180005200     MSVCRT:initializers.obj
 0002:00000208       __xc_z                     0000000180005208     MSVCRT:initializers.obj
 0002:00000210       __xi_a                     0000000180005210     MSVCRT:initializers.obj
 0002:00000220       __xi_z                     0000000180005220     MSVCRT:initializers.obj
 0002:00000228       __xl_a                     0000000180005228     MSVCRT:tlssup.obj
 0002:00000230       __xl_z                     0000000180005230     MSVCRT:tlssup.obj
 0002:00000238       __xp_a                     0000000180005238     MSVCRT:initializers.obj
 0002:00000240       __xp_z                     0000000180005240     MSVCRT:initializers.obj
 0002:00000248       __xt_a                     0000000180005248     MSVCRT:initializers.obj
 0002:00000250       __xt_z                     0000000180005250     MSVCRT:initializers.obj
 0002:00000260       g_refKindStr               0000000180005260     libobjfree002.obj
 0002:00000410       ??_C@_09BPLDFGCI@unknown_0@ 0000000180005410     libobjfree002.obj
 0002:00000420       ??_C@_0BL@FPNMECJD@JVMTI_HEAP_REFERENCE_CLASS@ 0000000180005420     libobjfree002.obj
 0002:00000440       ??_C@_0BL@FKGKKLNM@JVMTI_HEAP_REFERENCE_FIELD@ 0000000180005440     libobjfree002.obj
 0002:00000460       ??_C@_0CD@CAEHCFJF@JVMTI_HEAP_REFERENCE_ARRAY_ELEM@ 0000000180005460     libobjfree002.obj
 0002:00000488       ??_C@_0CC@DNEBMCNK@JVMTI_HEAP_REFERENCE_CLASS_LOAD@ 0000000180005488     libobjfree002.obj
 0002:000004b0       ??_C@_0BN@CJMIPEBB@JVMTI_HEAP_REFERENCE_SIGNERS@ 00000001800054b0     libobjfree002.obj
 0002:000004d0       ??_C@_0CH@HBOIDPEB@JVMTI_HEAP_REFERENCE_PROTECTION@ 00000001800054d0     libobjfree002.obj
 0002:000004f8       ??_C@_0BP@MDKGDGKL@JVMTI_HEAP_REFERENCE_INTERFACE@ 00000001800054f8     libobjfree002.obj
 0002:00000518       ??_C@_0CC@JJMIHNJH@JVMTI_HEAP_REFERENCE_STATIC_FIE@ 0000000180005518     libobjfree002.obj
 0002:00000540       ??_C@_0CD@IDHEEGID@JVMTI_HEAP_REFERENCE_CONSTANT_P@ 0000000180005540     libobjfree002.obj
 0002:00000568       ??_C@_0CA@EFFCHNG@JVMTI_HEAP_REFERENCE_SUPERCLASS@ 0000000180005568     libobjfree002.obj
 0002:00000588       ??_C@_0L@PCDFHGCJ@unknown_11@ 0000000180005588     libobjfree002.obj
 0002:00000598       ??_C@_0L@NJBICFOK@unknown_12@ 0000000180005598     libobjfree002.obj
 0002:000005a8       ??_C@_0L@MAADBEKL@unknown_13@ 00000001800055a8     libobjfree002.obj
 0002:000005b8       ??_C@_0L@IPECICGM@unknown_14@ 00000001800055b8     libobjfree002.obj
 0002:000005c8       ??_C@_0L@JGFJLDCN@unknown_15@ 00000001800055c8     libobjfree002.obj
 0002:000005d8       ??_C@_0L@LNHEOAOO@unknown_16@ 00000001800055d8     libobjfree002.obj
 0002:000005e8       ??_C@_0L@KEGPNBKP@unknown_17@ 00000001800055e8     libobjfree002.obj
 0002:000005f8       ??_C@_0L@CDPHMNGA@unknown_18@ 00000001800055f8     libobjfree002.obj
 0002:00000608       ??_C@_0L@DKOMPMCB@unknown_19@ 0000000180005608     libobjfree002.obj
 0002:00000618       ??_C@_0L@OJGIPJDB@unknown_20@ 0000000180005618     libobjfree002.obj
 0002:00000628       ??_C@_0CA@KAOFNDEM@JVMTI_HEAP_REFERENCE_JNI_GLOBAL@ 0000000180005628     libobjfree002.obj
 0002:00000648       ??_C@_0CC@HPFAJBK@JVMTI_HEAP_REFERENCE_SYSTEM_CLA@ 0000000180005648     libobjfree002.obj
 0002:00000670       ??_C@_0BN@FDEGFOHC@JVMTI_HEAP_REFERENCE_MONITOR@ 0000000180005670     libobjfree002.obj
 0002:00000690       ??_C@_0CB@HKIBCMAJ@JVMTI_HEAP_REFERENCE_STACK_LOCA@ 0000000180005690     libobjfree002.obj
 0002:000006b8       ??_C@_0BP@EAACMMOE@JVMTI_HEAP_REFERENCE_JNI_LOCAL@ 00000001800056b8     libobjfree002.obj
 0002:000006d8       ??_C@_0BM@IJDEOGOE@JVMTI_HEAP_REFERENCE_THREAD@ 00000001800056d8     libobjfree002.obj
 0002:000006f8       ??_C@_0BL@EDGPPKC@JVMTI_HEAP_REFERENCE_OTHER@ 00000001800056f8     libobjfree002.obj
 0002:00000714       ??_C@_04BCJPDBDA@Code@     0000000180005714     libobjfree002.obj
 0002:00000720       ??_C@_0BA@OCLMCFKC@LineNumberTable@ 0000000180005720     libobjfree002.obj
 0002:00000730       ??_C@_0BD@CPAEPILC@LocalVariableTable@ 0000000180005730     libobjfree002.obj
 0002:00000748       ??_C@_0BH@NMBDNHBD@LocalVariableTypeTable@ 0000000180005748     libobjfree002.obj
 0002:00000760       ??_C@_0O@HIHEEDNJ@StackMapTable@ 0000000180005760     libobjfree002.obj
 0002:00000770       ??_C@_0L@HCDIAMJG@?9?5?$CFs?0?5?$CFd?3?5@ 0000000180005770     libobjfree002.obj
 0002:00000780       ??_C@_0JI@HLPECLFI@?$CD?5?4?4?4?6?$CD?5ERROR?3?5too?5many?5complai@ 0000000180005780     libobjfree002.obj
 0002:00000820       ??_C@_0ED@JNEKCCOB@The?5following?5fake?5exception?5st@ 0000000180005820     libobjfree002.obj
 0002:00000868       ??_C@_0CN@FCNMDFBH@nsk?4share?4Fake_Exception_for_RU@ 0000000180005868     libobjfree002.obj
 0002:00000898       ??_C@_08PGFFNAEI@?$CI?$CFs?3?$CFd?$CJ?5@ 0000000180005898     libobjfree002.obj
 0002:000008a8       ??_C@_0DP@IENMAEGI@s?2test?2hotspot?2jtreg?2vmTestbase@ 00000001800058a8     libobjfree002.obj
 0002:000008e8       ??_C@_0BL@NDJLFFJB@?7at?5nsk_lvcomplain?$CI?$CFs?3?$CFd?$CJ?6@ 00000001800058e8     libobjfree002.obj
 0002:00000908       ??_C@_0BC@JOOKAFKF@?$CD?5ERROR?3?5?$CFs?0?5?$CFd?3?5@ 0000000180005908     libobjfree002.obj
 0002:00000920       ??_C@_09KJEAHMEH@?$CD?5ERROR?3?5@ 0000000180005920     libobjfree002.obj
 0002:0000092c       ??_C@_02GPIOPFAK@?$DO?$DO@ 000000018000592c     libobjfree002.obj
 0002:00000930       ??_C@_02FODMEDOG@?$DM?$DM@ 0000000180005930     libobjfree002.obj
 0002:00000934       ??_C@_02DJGKEECL@?4?4@     0000000180005934     libobjfree002.obj
 0002:00000938       ??_C@_0O@CJPGJOAF@?9?5?$CFs?0?5?$CFd?3?5?$CFs?5@ 0000000180005938     libobjfree002.obj
 0002:00000948       ??_C@_0CB@IAKPDOIC@?$CD?5?5?5verified?5assertion?5is?5FALSE@ 0000000180005948     libobjfree002.obj
 0002:00000970       ??_C@_0CO@LGONDEPD@stdout?3?5fflush?5failed?5?9?5err?$DN?$CFd?5@ 0000000180005970     libobjfree002.obj
 0002:000009a0       ??_C@_0CO@KBGKJPBD@stderr?3?5fflush?5failed?5?9?5err?$DN?$CFd?5@ 00000001800059a0     libobjfree002.obj
 0002:000009d0       ??_C@_0BB@JCNMKLLK@JVMTI_ERROR_NONE@ 00000001800059d0     libobjfree002.obj
 0002:000009e8       ??_C@_0BL@LDIMKLPH@JVMTI_ERROR_INVALID_THREAD@ 00000001800059e8     libobjfree002.obj
 0002:00000a08       ??_C@_0CB@PJFPAIKJ@JVMTI_ERROR_INVALID_THREAD_GROU@ 0000000180005a08     libobjfree002.obj
 0002:00000a30       ??_C@_0BN@LLMKHMNF@JVMTI_ERROR_INVALID_PRIORITY@ 0000000180005a30     libobjfree002.obj
 0002:00000a50       ??_C@_0CB@MBOFKAGB@JVMTI_ERROR_THREAD_NOT_SUSPENDE@ 0000000180005a50     libobjfree002.obj
 0002:00000a78       ??_C@_0BN@FABOLPBI@JVMTI_ERROR_THREAD_SUSPENDED@ 0000000180005a78     libobjfree002.obj
 0002:00000a98       ??_C@_0BN@FDGNOBJM@JVMTI_ERROR_THREAD_NOT_ALIVE@ 0000000180005a98     libobjfree002.obj
 0002:00000ab8       ??_C@_0BL@GOBIFKNJ@JVMTI_ERROR_INVALID_OBJECT@ 0000000180005ab8     libobjfree002.obj
 0002:00000ad8       ??_C@_0BK@FCMAJPPC@JVMTI_ERROR_INVALID_CLASS@ 0000000180005ad8     libobjfree002.obj
 0002:00000af8       ??_C@_0BP@IKLLBKEB@JVMTI_ERROR_CLASS_NOT_PREPARED@ 0000000180005af8     libobjfree002.obj
 0002:00000b18       ??_C@_0BN@KLPPLKG@JVMTI_ERROR_INVALID_METHODID@ 0000000180005b18     libobjfree002.obj
 0002:00000b38       ??_C@_0BN@BCEKOKND@JVMTI_ERROR_INVALID_LOCATION@ 0000000180005b38     libobjfree002.obj
 0002:00000b58       ??_C@_0BM@DFDGPME@JVMTI_ERROR_INVALID_FIELDID@ 0000000180005b58     libobjfree002.obj
 0002:00000b78       ??_C@_0BL@NELIEPEC@JVMTI_ERROR_NO_MORE_FRAMES@ 0000000180005b78     libobjfree002.obj
 0002:00000b98       ??_C@_0BJ@BDBECFDM@JVMTI_ERROR_OPAQUE_FRAME@ 0000000180005b98     libobjfree002.obj
 0002:00000bb8       ??_C@_0BK@MIIFNLOB@JVMTI_ERROR_TYPE_MISMATCH@ 0000000180005bb8     libobjfree002.obj
 0002:00000bd8       ??_C@_0BJ@HPCAOILC@JVMTI_ERROR_INVALID_SLOT@ 0000000180005bd8     libobjfree002.obj
 0002:00000bf8       ??_C@_0BG@CHILOPNI@JVMTI_ERROR_DUPLICATE@ 0000000180005bf8     libobjfree002.obj
 0002:00000c10       ??_C@_0BG@DIEMLHKM@JVMTI_ERROR_NOT_FOUND@ 0000000180005c10     libobjfree002.obj
 0002:00000c28       ??_C@_0BM@NHMCKHOB@JVMTI_ERROR_INVALID_MONITOR@ 0000000180005c28     libobjfree002.obj
 0002:00000c48       ??_C@_0BO@PPEDAJGL@JVMTI_ERROR_NOT_MONITOR_OWNER@ 0000000180005c48     libobjfree002.obj
 0002:00000c68       ??_C@_0BG@FCAIPEID@JVMTI_ERROR_INTERRUPT@ 0000000180005c68     libobjfree002.obj
 0002:00000c80       ??_C@_0CB@EGDBNKOI@JVMTI_ERROR_INVALID_CLASS_FORMA@ 0000000180005c80     libobjfree002.obj
 0002:00000ca8       ??_C@_0CG@DGKOGIAL@JVMTI_ERROR_CIRCULAR_CLASS_DEFI@ 0000000180005ca8     libobjfree002.obj
 0002:00000cd0       ??_C@_0BP@ICEALPKC@JVMTI_ERROR_FAILS_VERIFICATION@ 0000000180005cd0     libobjfree002.obj
 0002:00000cf0       ??_C@_0DC@JDACLMIO@JVMTI_ERROR_UNSUPPORTED_REDEFIN@ 0000000180005cf0     libobjfree002.obj
 0002:00000d28       ??_C@_0DE@GKDKNOMJ@JVMTI_ERROR_UNSUPPORTED_REDEFIN@ 0000000180005d28     libobjfree002.obj
 0002:00000d60       ??_C@_0BO@LAFKIOG@JVMTI_ERROR_INVALID_TYPESTATE@ 0000000180005d60     libobjfree002.obj
 0002:00000d80       ??_C@_0DH@INDGCLLB@JVMTI_ERROR_UNSUPPORTED_REDEFIN@ 0000000180005d80     libobjfree002.obj
 0002:00000db8       ??_C@_0DE@NHEOMMGI@JVMTI_ERROR_UNSUPPORTED_REDEFIN@ 0000000180005db8     libobjfree002.obj
 0002:00000df0       ??_C@_0CA@EKPNJOEP@JVMTI_ERROR_UNSUPPORTED_VERSION@ 0000000180005df0     libobjfree002.obj
 0002:00000e10       ??_C@_0BN@OFFMAHHL@JVMTI_ERROR_NAMES_DONT_MATCH@ 0000000180005e10     libobjfree002.obj
 0002:00000e30       ??_C@_0DN@HHBBLAKE@JVMTI_ERROR_UNSUPPORTED_REDEFIN@ 0000000180005e30     libobjfree002.obj
 0002:00000e70       ??_C@_0DO@HMBGBGNA@JVMTI_ERROR_UNSUPPORTED_REDEFIN@ 0000000180005e70     libobjfree002.obj
 0002:00000eb0       ??_C@_0BP@PBECGKHJ@JVMTI_ERROR_UNMODIFIABLE_CLASS@ 0000000180005eb0     libobjfree002.obj
 0002:00000ed0       ??_C@_0BK@CANILEHF@JVMTI_ERROR_NOT_AVAILABLE@ 0000000180005ed0     libobjfree002.obj
 0002:00000ef0       ??_C@_0CE@INJKMEFK@JVMTI_ERROR_MUST_POSSESS_CAPABI@ 0000000180005ef0     libobjfree002.obj
 0002:00000f18       ??_C@_0BJ@LBFPFPDM@JVMTI_ERROR_NULL_POINTER@ 0000000180005f18     libobjfree002.obj
 0002:00000f38       ??_C@_0BP@CHJPNNEM@JVMTI_ERROR_ABSENT_INFORMATION@ 0000000180005f38     libobjfree002.obj
 0002:00000f58       ??_C@_0BP@OMFMNLC@JVMTI_ERROR_INVALID_EVENT_TYPE@ 0000000180005f58     libobjfree002.obj
 0002:00000f78       ??_C@_0BN@BIBNPHHO@JVMTI_ERROR_ILLEGAL_ARGUMENT@ 0000000180005f78     libobjfree002.obj
 0002:00000f98       ??_C@_0BK@KKNDHDCE@JVMTI_ERROR_NATIVE_METHOD@ 0000000180005f98     libobjfree002.obj
 0002:00000fb8       ??_C@_0BK@PMKCFHAE@JVMTI_ERROR_OUT_OF_MEMORY@ 0000000180005fb8     libobjfree002.obj
 0002:00000fd8       ??_C@_0BK@NNJBDMNB@JVMTI_ERROR_ACCESS_DENIED@ 0000000180005fd8     libobjfree002.obj
 0002:00000ff8       ??_C@_0BI@GHECLMNC@JVMTI_ERROR_WRONG_PHASE@ 0000000180005ff8     libobjfree002.obj
 0002:00001010       ??_C@_0BF@OLIHJOII@JVMTI_ERROR_INTERNAL@ 0000000180006010     libobjfree002.obj
 0002:00001028       ??_C@_0BO@EOHGKJHI@JVMTI_ERROR_UNATTACHED_THREAD@ 0000000180006028     libobjfree002.obj
 0002:00001048       ??_C@_0CA@LKHFDACL@JVMTI_ERROR_INVALID_ENVIRONMENT@ 0000000180006048     libobjfree002.obj
 0002:00001068       ??_C@_0BA@MMFHLOKK@?$DMunknown?5error?$DO@ 0000000180006068     libobjfree002.obj
 0002:00001078       ??_C@_0CF@CBHOKDB@throwable?5?$DN?5jni?9?$DOExceptionOccur@ 0000000180006078     libobjfree002.obj
 0002:000010a0       ??_C@_03OFAPEBGM@?$CFs?6@  00000001800060a0     libobjfree002.obj
 0002:000010a8       ??_C@_0DM@LPIGEGNJ@s?2test?2hotspot?2jtreg?2vmTestbase@ 00000001800060a8     libobjfree002.obj
 0002:000010e8       ??_C@_0CC@NFCNPEPK@Exception?5in?5JNI?5call?5?$CIcleared?$CJ@ 00000001800060e8     libobjfree002.obj
 0002:00001110       ??_C@_0BJ@IBAKFIKF@jni?9?$DOExceptionDescribe?$CI?$CJ@ 0000000180006110     libobjfree002.obj
 0002:00001130       ??_C@_0BG@GGKALKMH@jni?9?$DOExceptionClear?$CI?$CJ@ 0000000180006130     libobjfree002.obj
 0002:00001148       ??_C@_0CF@JMGFGJLJ@?$CD?5?5?5verified?5JNI?5assertion?5is?5F@ 0000000180006148     libobjfree002.obj
 0002:00001170       ??_C@_07KBAMPNJK@verbose@  0000000180006170     libobjfree002.obj
 0002:00001178       ??_C@_0DN@PKJBOLAP@nsk_jvmti_parseOptions?$CI?$CJ?3?5unexp@ 0000000180006178     libobjfree002.obj
 0002:000011b8       ??_C@_05IMBNNINJ@trace@    00000001800061b8     libobjfree002.obj
 0002:000011c0       ??_C@_0DD@BJKGNDMB@nsk_jvmti_parseOptions?$CI?$CJ?3?5no?5va@ 00000001800061c0     libobjfree002.obj
 0002:000011f4       ??_C@_04CGFJFPFD@none@     00000001800061f4     libobjfree002.obj
 0002:000011fc       ??_C@_06BMELKFMA@before@   00000001800061fc     libobjfree002.obj
 0002:00001204       ??_C@_05CMKPCFDK@after@    0000000180006204     libobjfree002.obj
 0002:0000120c       ??_C@_03NFKEKGGK@all@      000000018000620c     libobjfree002.obj
 0002:00001210       ??_C@_0DM@NDNJGJKE@nsk_jvmti_parseOptions?$CI?$CJ?3?5uexpe@ 0000000180006210     libobjfree002.obj
 0002:00001250       ??_C@_08NBBJKJO@waittime@  0000000180006250     libobjfree002.obj
 0002:00001260       ??_C@_0DO@CMHGAOHC@nsk_jvmti_parseOptions?$CI?$CJ?3?5not?5i@ 0000000180006260     libobjfree002.obj
 0002:000012a0       ??_C@_0DL@LNMPBDLN@nsk_jvmti_parseOptions?$CI?$CJ?3?5negat@ 00000001800062a0     libobjfree002.obj
 0002:000012e0       ??_C@_0DA@GMFJNOJH@nsk_jvmti_parseOptions?$CI?$CJ?3?5unkno@ 00000001800062e0     libobjfree002.obj
 0002:00001310       ??_C@_0CO@CCIAMEAN@nsk_jvmti_parseOptions?$CI?$CJ?3?5found@ 0000000180006310     libobjfree002.obj
 0002:00001340       ??_C@_0CJ@OEGPCGDL@nsk_jvmti_parseOptions?$CI?$CJ?3?5out?5o@ 0000000180006340     libobjfree002.obj
 0002:00001370       ??_C@_0DI@NMBHPGGF@nsk_jvmti_parseOptions?$CI?$CJ?3?5too?5m@ 0000000180006370     libobjfree002.obj
 0002:000013a8       ??_C@_03POGCGECB@?5?0?$HO@ 00000001800063a8     libobjfree002.obj
 0002:000013b0       ??_C@_0CB@MLNJNCLJ@?5?5jvmti?5error?3?5code?$DN?$CFd?0?5name?$DN?$CFs@ 00000001800063b0     libobjfree002.obj
 0002:000013d8       ??_C@_0CD@OHBGDKMK@?$CD?5?5?5jvmti?5error?3?5code?$DN?$CFd?0?5name?$DN@ 00000001800063d8     libobjfree002.obj
 0002:00001400       ??_C@_0CG@JNNCGPHB@?$CD?5?5?5error?5expected?3?5code?$DN?$CFd?0?5na@ 0000000180006400     libobjfree002.obj
 0002:00001430       ??_C@_0EB@IMGKPCGE@?$CIstr_obj?5?$DN?5jni?9?$DONewStringUTF?$CIco@ 0000000180006430     libobjfree002.obj
 0002:00001480       ??_C@_0EA@HFOGGBCC@s?2test?2hotspot?2jtreg?2vmTestbase@ 0000000180006480     libobjfree002.obj
 0002:000014c0       ??_C@_05KKCIMGE@error@     00000001800064c0     libobjfree002.obj
 0002:000014c8       ??_C@_0BD@HGNAOMCP@agent_data_monitor@ 00000001800064c8     libobjfree002.obj
 0002:000014e0       ??_C@_0EB@OGCLGKLN@javaVM?9?$DOGetEnv?$CI?$CIvoid?5?$CK?$CK?$CJ?$CGjvmti_@ 00000001800064e0     libobjfree002.obj
 0002:00001530       ??_C@_0EA@PNBCDMOA@s?2test?2hotspot?2jtreg?2vmTestbase@ 0000000180006530     libobjfree002.obj
 0002:00001570       ??_C@_0CI@DDPIFBGM@init_agent_data?$CIjvmti_env?0?5?$CGage@ 0000000180006570     libobjfree002.obj
 0002:00001598       ??_C@_0DI@ILAHDLMP@?$CI?$CKagentThreadProc?$CJ?$CIjvmti_env?0?5a@ 0000000180006598     libobjfree002.obj
 0002:000015d0       ??_C@_0BD@KDBALNLB@JVMTI?5agent?5thread@ 00000001800065d0     libobjfree002.obj
 0002:000015e8       ??_C@_0BB@NOKBFPFO@java?1lang?1Thread@ 00000001800065e8     libobjfree002.obj
 0002:000015fc       ??_C@_06FALKBLGB@?$DMinit?$DO@ 00000001800065fc     libobjfree002.obj
 0002:00001608       ??_C@_0BG@IKDDPPGD@?$CILjava?1lang?1String?$DL?$CJV@ 0000000180006608     libobjfree002.obj
 0002:00001620       ??_C@_0EB@IFJBFEKC@?$CIthreadClass?5?$DN?5jni_env?9?$DOFindCla@ 0000000180006620     libobjfree002.obj
 0002:00001670       ??_C@_0GF@FGFIBKKL@?$CIthreadCtor?5?$DN?5jni_env?9?$DOGetMetho@ 0000000180006670     libobjfree002.obj
 0002:000016d8       ??_C@_0DN@NCPDJLOG@?$CIthreadName?5?$DN?5jni_env?9?$DONewStrin@ 00000001800066d8     libobjfree002.obj
 0002:00001720       ??_C@_0FE@PFKODBGC@?$CIthreadObject?5?$DN?5jni_env?9?$DONewObj@ 0000000180006720     libobjfree002.obj
 0002:00001780       ??_C@_0ED@HOBAHHJI@?$CIthreadGlobalRef?5?$DN?5jni_env?9?$DONew@ 0000000180006780     libobjfree002.obj
 0002:000017d0       ??_C@_0FN@HNJJAHFC@jvmti_env?9?$DORunAgentThread?$CIagent@ 00000001800067d0     libobjfree002.obj
 0002:00001830       ??_C@_0EA@MOJDNKDF@Debuggee?5status?5sync?5aborted?5be@ 0000000180006830     libobjfree002.obj
 0002:00001870       ??_C@_0EA@EEOEJAEN@status?5?$DN?5syncDebuggeeStatus?$CIjni@ 0000000180006870     libobjfree002.obj
 0002:000018b0       ??_C@_0BL@JBCFNBMB@nsk_jvmti_resetAgentData?$CI?$CJ@ 00000001800068b0     libobjfree002.obj
 0002:000018d0       ??_C@_0EL@LPBEELIP@s?2test?2hotspot?2jtreg?2vmTestbase@ 00000001800068d0     libobjfree002.obj
 0002:00001920       ??_C@_0CK@JDAMFDMJ@jvmti?9?$DOSetTag?$CIo?0?5tag?$CJ?5?$DN?$DN?5JVMTI_@ 0000000180006920     libobjfree002.obj
 0002:00001950       ??_C@_0CC@DAMNHKNI@Can?8t?5set?5tag?5?$CFli?5for?5object?5?$CFl@ 0000000180006950     libobjfree002.obj
 0002:00001978       ??_C@_0DL@HAJPNKEF@jvmti?9?$DOGetObjectHashCode?$CIo?0?5?$CGha@ 0000000180006978     libobjfree002.obj
 0002:000019b8       ??_C@_0BL@JFPIEOBF@Can?8t?5get?5hash?5object?5?$CFlx?6@ 00000001800069b8     libobjfree002.obj
 0002:000019d8       ??_C@_0BG@DICPHBKN@setTag?3?5?$CF08x?5?$DM?9?5?$CF?53li@ 00000001800069d8     libobjfree002.obj
 0002:000019f0       ??_C@_0DH@FCEEBDMJ@?$CIs?5?$DN?5jni?9?$DOGetStringUTFChars?$CIsIn@ 00000001800069f0     libobjfree002.obj
 0002:00001a28       ??_C@_0BJ@OKKGHDCN@Can?8t?5get?5string?5at?5?$CF?$CDp?6@ 0000000180006a28     libobjfree002.obj
 0002:00001a48       ??_C@_0BP@EKFLGGFJ@Can?8t?5get?5string?5at?5?$CF?$CDp?3?5null?6@ 0000000180006a48     libobjfree002.obj
 0002:00001a68       ??_C@_06ICODBHCL@?5?1?1?5?$CFs@ 0000000180006a68     libobjfree002.obj
 0002:00001a70       ??_C@_0DB@KGFPLEGO@?$CIr?5?$DN?5jvmti?9?$DOGetTag?$CIo?0?5?$CGtag?$CJ?$CJ?5?$DN?$DN@ 0000000180006a70     libobjfree002.obj
 0002:00001aa8       ??_C@_0CO@PDAGBCGJ@Can?8t?5GetTag?5for?5object?5?$CFlx?4?5Re@ 0000000180006aa8     libobjfree002.obj
 0002:00001ad8       ??_C@_0CH@HPEODOHC@TEST_BUG?3?5Max?4?5number?5of?5refs?5r@ 0000000180006ad8     libobjfree002.obj
 0002:00001b00       ??_C@_0DI@PHFCABIM@?$CIr?5?$DN?5jvmti?9?$DOGetTag?$CIfrom?0?5?$CGtagFr@ 0000000180006b00     libobjfree002.obj
 0002:00001b38       ??_C@_0DI@MDEGFNKD@TEST_BUG?3?5Can?8t?5GetTag?5for?5obje@ 0000000180006b38     libobjfree002.obj
 0002:00001b70       ??_C@_0DE@MLELJAHM@?$CIr?5?$DN?5jvmti?9?$DOGetTag?$CIto?0?5?$CGtagTo?$CJ?$CJ@ 0000000180006b70     libobjfree002.obj
 0002:00001ba8       ??_C@_0CA@NFFMLHN@?$CFs?3?5creating?5a?5raw?5monitor?5?4?4?4?6@ 0000000180006ba8     libobjfree002.obj
 0002:00001bd0       ??_C@_0EP@FGBFMJHI@s?2test?2hotspot?2jtreg?2vmTestbase@ 0000000180006bd0     libobjfree002.obj
 0002:00001c20       ??_C@_0CN@GMOGLIIN@jvmti_env?9?$DOCreateRawMonitor?$CI?$CC_l@ 0000000180006c20     libobjfree002.obj
 0002:00001c50       ??_C@_05EAPKFOHC@_lock@    0000000180006c50     libobjfree002.obj
 0002:00001c58       ??_C@_0DC@BFAML@TEST?5FAILED?3?5?$CFs?3?5unable?5to?5crea@ 0000000180006c58     libobjfree002.obj
 0002:00001c90       ??_C@_0CH@ELPNCNMM@CHECK?5PASSED?3?5?$CFs?3?5raw?5monitor?5c@ 0000000180006c90     libobjfree002.obj
 0002:00001cb8       ??_C@_0CC@KPNBIBOK@?$CFs?3?5entering?5the?5raw?5monitor?5?4?4@ 0000000180006cb8     libobjfree002.obj
 0002:00001ce0       ??_C@_0CC@LICKJMEG@jvmti_env?9?$DORawMonitorEnter?$CI_loc@ 0000000180006ce0     libobjfree002.obj
 0002:00001d08       ??_C@_0DD@ILNKINHA@TEST?5FAILED?3?5?$CFs?3?5unable?5to?5ente@ 0000000180006d08     libobjfree002.obj
 0002:00001d40       ??_C@_0CL@HOBMHNLB@CHECK?5PASSED?3?5?$CFs?3?5the?5raw?5monit@ 0000000180006d40     libobjfree002.obj
 0002:00001d70       ??_C@_0CB@CKCFLCHC@?$CFs?3?5waiting?5the?5raw?5monitor?5?4?4?4@ 0000000180006d70     libobjfree002.obj
 0002:00001d98       ??_C@_0CM@JCJEGOIK@jvmti_env?9?$DORawMonitorWait?$CI_lock@ 0000000180006d98     libobjfree002.obj
 0002:00001dc8       ??_C@_0DC@HEFDLADG@TEST?5FAILED?3?5?$CFs?3?5unable?5to?5wait@ 0000000180006dc8     libobjfree002.obj
 0002:00001e00       ??_C@_0CK@FALIEPOD@CHECK?5PASSED?3?5?$CFs?3?5the?5raw?5monit@ 0000000180006e00     libobjfree002.obj
 0002:00001e30       ??_C@_0DO@LEDIEDGM@?$CFs?3?5notifying?5a?5single?5thread?5w@ 0000000180006e30     libobjfree002.obj
 0002:00001e70       ??_C@_0CD@MCEJJMHC@jvmti_env?9?$DORawMonitorNotify?$CI_lo@ 0000000180006e70     libobjfree002.obj
 0002:00001e98       ??_C@_0DC@NDHFJDDN@TEST?5FAILED?3?5?$CFs?3?5unable?5to?5noti@ 0000000180006e98     libobjfree002.obj
 0002:00001ed0       ??_C@_0CK@MNPOBPIB@CHECK?5PASSED?3?5?$CFs?3?5single?5thread@ 0000000180006ed0     libobjfree002.obj
 0002:00001f00       ??_C@_0DK@BAPFBNKN@?$CFs?3?5notifying?5all?5threads?5waiti@ 0000000180006f00     libobjfree002.obj
 0002:00001f40       ??_C@_0CG@ICKGGLBM@jvmti_env?9?$DORawMonitorNotifyAll?$CI@ 0000000180006f40     libobjfree002.obj
 0002:00001f68       ??_C@_0DA@KDBFDPJM@TEST?5FAILED?3?5?$CFs?3?5unable?5to?5noti@ 0000000180006f68     libobjfree002.obj
 0002:00001f98       ??_C@_0CI@LELHIBGI@CHECK?5PASSED?3?5?$CFs?3?5all?5threads?5n@ 0000000180006f98     libobjfree002.obj
 0002:00001fc0       ??_C@_0CB@HNKHEJBK@?$CFs?3?5exiting?5the?5raw?5monitor?5?4?4?4@ 0000000180006fc0     libobjfree002.obj
 0002:00001fe8       ??_C@_0CB@FEMOEOEG@jvmti_env?9?$DORawMonitorExit?$CI_lock@ 0000000180006fe8     libobjfree002.obj
 0002:00002010       ??_C@_0DC@JPCLONBC@TEST?5FAILED?3?5?$CFs?3?5unable?5to?5exit@ 0000000180007010     libobjfree002.obj
 0002:00002048       ??_C@_0CK@JMGAKAKI@CHECK?5PASSED?3?5?$CFs?3?5the?5raw?5monit@ 0000000180007048     libobjfree002.obj
 0002:00002078       ??_C@_0CE@KLCCECNE@?$CFs?3?5destroying?5the?5raw?5monitor?5@ 0000000180007078     libobjfree002.obj
 0002:000020a0       ??_C@_0CE@LMOOLBIH@jvmti_env?9?$DODestroyRawMonitor?$CI_l@ 00000001800070a0     libobjfree002.obj
 0002:000020c8       ??_C@_0DC@PKLDHPCH@TEST?5FAILED?3?5?$CFs?3?5unable?5to?5dest@ 00000001800070c8     libobjfree002.obj
 0002:00002100       ??_C@_0CN@NBOLIIFJ@CHECK?5PASSED?3?5?$CFs?3?5the?5raw?5monit@ 0000000180007100     libobjfree002.obj
 0002:00002130       ??_C@_0BL@EDKNLHDL@?$CFs?3?5allocating?5memory?5?4?4?4?6@ 0000000180007130     libobjfree002.obj
 0002:00002150       ??_C@_0CE@DFLKJLND@jvmti_env?9?$DOAllocate?$CIMEM_SIZE?0?5?$CG@ 0000000180007150     libobjfree002.obj
 0002:00002178       ??_C@_0CN@BDGANOPB@TEST?5FAILED?3?5?$CFs?3?5unable?5to?5allo@ 0000000180007178     libobjfree002.obj
 0002:000021a8       ??_C@_0DK@KLGPKMFP@CHECK?5PASSED?3?5?$CFs?3?5memory?5has?5be@ 00000001800071a8     libobjfree002.obj
 0002:000021e8       ??_C@_0BN@EKKCBNLG@?$CFs?3?5deallocating?5memory?5?4?4?4?6@ 00000001800071e8     libobjfree002.obj
 0002:00002208       ??_C@_0BL@KHDPKCEF@jvmti_env?9?$DODeallocate?$CImem?$CJ@ 0000000180007208     libobjfree002.obj
 0002:00002228       ??_C@_0CP@PGMPPCAM@TEST?5FAILED?3?5?$CFs?3?5unable?5to?5deal@ 0000000180007228     libobjfree002.obj
 0002:00002258       ??_C@_0DM@ICINEJJJ@CHECK?5PASSED?3?5?$CFs?3?5memory?5has?5be@ 0000000180007258     libobjfree002.obj
 0002:00002298       ??_C@_0DD@MOEHFALM@?$CFs?3?5setting?5an?5environment?5loca@ 0000000180007298     libobjfree002.obj
 0002:000022d0       ??_C@_0DL@NKBHLEAC@jvmti_env?9?$DOSetEnvironmentLocalS@ 00000001800072d0     libobjfree002.obj
 0002:00002310       ??_C@_0DO@KKDCNODO@TEST?5FAILED?3?5?$CFs?3?5unable?5to?5set?5@ 0000000180007310     libobjfree002.obj
 0002:00002350       ??_C@_0EH@DDHOCPGA@CHECK?5PASSED?3?5?$CFs?3?5environment?5l@ 0000000180007350     libobjfree002.obj
 0002:00002398       ??_C@_0CO@MCEDAAIL@?$CFs?3?5getting?5an?5environment?5loca@ 0000000180007398     libobjfree002.obj
 0002:000023c8       ??_C@_0DO@NNMJNLPF@jvmti_env?9?$DOGetEnvironmentLocalS@ 00000001800073c8     libobjfree002.obj
 0002:00002408       ??_C@_0DO@GNFCMJNH@TEST?5FAILED?3?5?$CFs?3?5unable?5to?5get?5@ 0000000180007408     libobjfree002.obj
 0002:00002450       ??_C@_0GK@CNDCICHK@TEST?5FAILED?3?5?$CFs?3?5obtained?5an?5en@ 0000000180007450     libobjfree002.obj
 0002:000024c0       ??_C@_0EI@BOJGAMEK@CHECK?5PASSED?3?5?$CFs?3?5environment?5l@ 00000001800074c0     libobjfree002.obj
 0002:00002508       ??_C@_0CA@MBAKPDCM@?$DO?$DO?$DO?$DO?5ObjectFree?5event?5received?6@ 0000000180007508     libobjfree002.obj
 0002:00002530       ??_C@_0EN@MLNAAAOM@TEST?5FAILED?3?5unexpected?5ObjectF@ 0000000180007530     libobjfree002.obj
 0002:00002580       ??_C@_0FH@GCMMAMBP@CHECK?5PASSED?3?5ObjectFree?5event?5@ 0000000180007580     libobjfree002.obj
 0002:000025d8       ??_C@_0L@DPGCJIOK@ObjectFree@ 00000001800075d8     libobjfree002.obj
 0002:000025e4       ??_C@_06FHLMFHLD@?$DM?$DM?$DM?$DM?6?6@ 00000001800075e4     libobjfree002.obj
 0002:000025f0       ??_C@_0BI@OPPGFBGD@VMDeath?5event?5received?6@ 00000001800075f0     libobjfree002.obj
 0002:00002610       ??_C@_0ED@LANFDPME@?6Warning?3?5no?5ObjectFree?5events?5@ 0000000180007610     libobjfree002.obj
 0002:00002658       ??_C@_0CG@IIOOGPCH@Setting?5the?5tag?5?$CC?$CFld?$CC?5for?5objec@ 0000000180007658     libobjfree002.obj
 0002:00002680       ??_C@_0CF@GPDJDLMJ@jvmti?9?$DOSetTag?$CIobjToTag?0?5?$CIjlong?$CJ@ 0000000180007680     libobjfree002.obj
 0002:000026a8       ??_C@_0CP@NDBIFLOB@TEST?5FAILED?3?5unable?5to?5set?5tag?5@ 00000001800076a8     libobjfree002.obj
 0002:000026d8       ??_C@_0CC@CPFDHHGP@Skipping?5object?5?$CD?$CFd?5from?5taggin@ 00000001800076d8     libobjfree002.obj
 0002:00002700       ??_C@_0CA@MNKGCBCG@nsk_jvmti_parseOptions?$CIoptions?$CJ@ 0000000180007700     libobjfree002.obj
 0002:00002720       ??_C@_0DN@MIAMNFPH@?$CIjvmti?5?$DN?5nsk_jvmti_createJVMTIE@ 0000000180007720     libobjfree002.obj
 0002:00002760       ??_C@_0BO@DBKDIPGD@jvmti?9?$DOAddCapabilities?$CI?$CGcaps?$CJ@ 0000000180007760     libobjfree002.obj
 0002:00002780       ??_C@_0BO@IAKFILDF@jvmti?9?$DOGetCapabilities?$CI?$CGcaps?$CJ@ 0000000180007780     libobjfree002.obj
 0002:000027a0       ??_C@_0DO@LDOBNMIH@Warning?3?5generation?5of?5object?5f@ 00000001800077a0     libobjfree002.obj
 0002:000027e0       ??_C@_0CN@GEOKBLEG@Warning?3?5tagging?5objects?5is?5not@ 00000001800077e0     libobjfree002.obj
 0002:00002810       ??_C@_0BN@HGIKGGD@setting?5event?5callbacks?5?4?4?4?6@ 0000000180007810     libobjfree002.obj
 0002:00002830       ??_C@_0DI@NJCFGEGC@jvmti?9?$DOSetEventCallbacks?$CI?$CGcallb@ 0000000180007830     libobjfree002.obj
 0002:00002868       ??_C@_0DI@LEFDPPF@setting?5event?5callbacks?5done?6en@ 0000000180007868     libobjfree002.obj
 0002:000028a0       ??_C@_0EN@OLHGIFGG@jvmti?9?$DOSetEventNotificationMode@ 00000001800078a0     libobjfree002.obj
 0002:000028f0       ??_C@_0FA@KLKMFDPK@jvmti?9?$DOSetEventNotificationMode@ 00000001800078f0     libobjfree002.obj
 0002:00002940       ??_C@_0BL@GBOGNFCP@enabling?5the?5events?5done?6?6@ 0000000180007940     libobjfree002.obj
 0002:00002970       ??_C@_1EC@JIJBPKFM@?$AAa?$AAp?$AAi?$AA?9?$AAm?$AAs?$AA?9?$AAw?$AAi?$AAn?$AA?9?$AAc?$AAo?$AAr?$AAe@ 0000000180007970     MSVCRT:thread_safe_statics.obj
 0002:000029b8       ??_C@_1BK@MGMFAEKH@?$AAk?$AAe?$AAr?$AAn?$AAe?$AAl?$AA3?$AA2?$AA?4?$AAd?$AAl?$AAl@ 00000001800079b8     MSVCRT:thread_safe_statics.obj
 0002:000029d8       ??_C@_0BJ@JEBJOJFJ@SleepConditionVariableCS@ 00000001800079d8     MSVCRT:thread_safe_statics.obj
 0002:000029f8       ??_C@_0BJ@PGPPEPCC@WakeAllConditionVariable@ 00000001800079f8     MSVCRT:thread_safe_statics.obj
 0002:00002a18       _pDefaultRawDllMain        0000000180007a18     MSVCRT:dll_dllmain.obj
 0002:00002a18       _pRawDllMain               0000000180007a18     MSVCRT:dll_dllmain.obj
 0002:00002a20       __xmm@ffffffffffffffffffffffffffffffff 0000000180007a20     MSVCRT:utility.obj
 0002:00002a30       _load_config_used          0000000180007a30     MSVCRT:loadcfg.obj
 0002:00002c00       _tls_used                  0000000180007c00     MSVCRT:tlssup.obj
 0002:00002c28       __volatile_metadata        0000000180007c28     <linker-defined>
 0002:00003040       __rtc_iaa                  0000000180008040     MSVCRT:initsect.obj
 0002:00003048       __rtc_izz                  0000000180008048     MSVCRT:initsect.obj
 0002:00003050       __rtc_taa                  0000000180008050     MSVCRT:initsect.obj
 0002:00003058       __rtc_tzz                  0000000180008058     MSVCRT:initsect.obj
 0002:00003060       _tls_start                 0000000180008060     MSVCRT:tlssup.obj
 0002:00003064       _Init_thread_epoch         0000000180008064     MSVCRT:thread_safe_statics.obj
 0002:00003068       _tls_end                   0000000180008068     MSVCRT:tlssup.obj
 0002:000037a0       __IMPORT_DESCRIPTOR_KERNEL32 00000001800087a0     kernel32:KERNEL32.dll
 0002:000037b4       __IMPORT_DESCRIPTOR_VCRUNTIME140 00000001800087b4     vcruntime:VCRUNTIME140.dll
 0002:000037c8       __IMPORT_DESCRIPTOR_api-ms-win-crt-heap-l1-1-0 00000001800087c8     ucrt:api-ms-win-crt-heap-l1-1-0.dll
 0002:000037dc       __IMPORT_DESCRIPTOR_api-ms-win-crt-runtime-l1-1-0 00000001800087dc     ucrt:api-ms-win-crt-runtime-l1-1-0.dll
 0002:000037f0       __IMPORT_DESCRIPTOR_api-ms-win-crt-convert-l1-1-0 00000001800087f0     ucrt:api-ms-win-crt-convert-l1-1-0.dll
 0002:00003804       __IMPORT_DESCRIPTOR_api-ms-win-crt-stdio-l1-1-0 0000000180008804     ucrt:api-ms-win-crt-stdio-l1-1-0.dll
 0002:00003818       __IMPORT_DESCRIPTOR_api-ms-win-crt-string-l1-1-0 0000000180008818     ucrt:api-ms-win-crt-string-l1-1-0.dll
 0002:0000382c       __NULL_IMPORT_DESCRIPTOR   000000018000882c     kernel32:KERNEL32.dll
 0003:00000030       _Init_global_epoch         0000000180009030     MSVCRT:thread_safe_statics.obj
 0003:00000040       __security_cookie          0000000180009040     MSVCRT:gs_cookie.obj
 0003:00000048       __security_cookie_complement 0000000180009048     MSVCRT:gs_cookie.obj
 0003:00000050       __scrt_native_dllmain_reason 0000000180009050     MSVCRT:utility.obj
 0003:00000058       __isa_available            0000000180009058     MSVCRT:cpu_disp.obj
 0003:0000005c       __isa_enabled              000000018000905c     MSVCRT:cpu_disp.obj
 0003:00000060       __memset_fast_string_threshold 0000000180009060     MSVCRT:cpu_disp.obj
 0003:00000068       __memset_nt_threshold      0000000180009068     MSVCRT:cpu_disp.obj
 0003:00000070       __scrt_ucrt_dll_is_in_use  0000000180009070     MSVCRT:ucrt_stubs.obj
 0003:00000080       g_wrongHeapCallbacks       0000000180009080     libobjfree002.obj
 0003:00000100       g_szTagInfo                0000000180009100     libobjfree002.obj
 0003:00002040       g_tagFlags                 000000018000b040     libobjfree002.obj
 0003:00002428       g_refsToVerifyCnt          000000018000b428     libobjfree002.obj
 0003:0000242c       g_fakeUserData             000000018000b42c     libobjfree002.obj
 0003:00002430       g_tagVisitCount            000000018000b430     libobjfree002.obj
 0003:000033d0       g_refsToVerify             000000018000c3d0     libobjfree002.obj
 0003:0001aad0       g_userDataError            0000000180023ad0     libobjfree002.obj
 0003:0001aad8       mem                        0000000180023ad8     libobjfree002.obj
 0003:0001b1d0       ?_OptionsStorage@?1??__local_stdio_printf_options@@9@4_KA 00000001800241d0     libobjfree002.obj
 0003:0001b798       _tls_index                 0000000180024798     MSVCRT:tlssup.obj
 0003:0001b7a0       __scrt_current_native_startup_state 00000001800247a0     MSVCRT:utility.obj
 0003:0001b7a8       __scrt_native_startup_lock 00000001800247a8     MSVCRT:utility.obj
 0003:0001b7e8       __scrt_debugger_hook_flag  00000001800247e8     MSVCRT:utility_desktop.obj
 0003:0001b7f0       ?__type_info_root_node@@3U__type_info_node@@A 00000001800247f0     MSVCRT:tncleanup.obj
 0003:0001b800       ?_OptionsStorage@?1??__local_stdio_scanf_options@@9@4_KA 0000000180024800     MSVCRT:default_local_stdio_options.obj
 0003:0001b808       __favor                    0000000180024808     MSVCRT:cpu_disp.obj
 0003:0001b810       __dyn_tls_init_callback    0000000180024810     <common>

 entry point at        0001:000032a0

 Static symbols

 0000:fffd9000       .debug$S                   0000000180000000     objfree002.exp
 0000:fffd9000       .debug$S                   0000000180000000     vcruntime:VCRUNTIME140.dll
 0000:fffd9000       .debug$S                   0000000180000000     vcruntime:VCRUNTIME140.dll
 0000:fffd9000       .debug$S                   0000000180000000     vcruntime:VCRUNTIME140.dll
 0000:fffd9000       .debug$S                   0000000180000000     vcruntime:VCRUNTIME140.dll
 0000:fffd9000       .debug$S                   0000000180000000     vcruntime:VCRUNTIME140.dll
 0000:fffd9000       .debug$S                   0000000180000000     vcruntime:VCRUNTIME140.dll
 0000:fffd9000       .debug$S                   0000000180000000     vcruntime:VCRUNTIME140.dll
 0000:fffd9000       .debug$S                   0000000180000000     ucrt:api-ms-win-crt-convert-l1-1-0.dll
 0000:fffd9000       .debug$S                   0000000180000000     ucrt:api-ms-win-crt-heap-l1-1-0.dll
 0000:fffd9000       .debug$S                   0000000180000000     ucrt:api-ms-win-crt-heap-l1-1-0.dll
 0000:fffd9000       .debug$S                   0000000180000000     ucrt:api-ms-win-crt-heap-l1-1-0.dll
 0000:fffd9000       .debug$S                   0000000180000000     ucrt:api-ms-win-crt-heap-l1-1-0.dll
 0000:fffd9000       .debug$S                   0000000180000000     ucrt:api-ms-win-crt-runtime-l1-1-0.dll
 0000:fffd9000       .debug$S                   0000000180000000     ucrt:api-ms-win-crt-runtime-l1-1-0.dll
 0000:fffd9000       .debug$S                   0000000180000000     ucrt:api-ms-win-crt-runtime-l1-1-0.dll
 0000:fffd9000       .debug$S                   0000000180000000     ucrt:api-ms-win-crt-runtime-l1-1-0.dll
 0000:fffd9000       .debug$S                   0000000180000000     ucrt:api-ms-win-crt-runtime-l1-1-0.dll
 0000:fffd9000       .debug$S                   0000000180000000     ucrt:api-ms-win-crt-runtime-l1-1-0.dll
 0000:fffd9000       .debug$S                   0000000180000000     ucrt:api-ms-win-crt-runtime-l1-1-0.dll
 0000:fffd9000       .debug$S                   0000000180000000     ucrt:api-ms-win-crt-runtime-l1-1-0.dll
 0000:fffd9000       .debug$S                   0000000180000000     ucrt:api-ms-win-crt-runtime-l1-1-0.dll
 0000:fffd9000       .debug$S                   0000000180000000     ucrt:api-ms-win-crt-runtime-l1-1-0.dll
 0000:fffd9000       .debug$S                   0000000180000000     ucrt:api-ms-win-crt-runtime-l1-1-0.dll
 0000:fffd9000       .debug$S                   0000000180000000     ucrt:api-ms-win-crt-runtime-l1-1-0.dll
 0000:fffd9000       .debug$S                   0000000180000000     ucrt:api-ms-win-crt-runtime-l1-1-0.dll
 0000:fffd9000       .debug$S                   0000000180000000     ucrt:api-ms-win-crt-runtime-l1-1-0.dll
 0000:fffd9000       .debug$S                   0000000180000000     ucrt:api-ms-win-crt-runtime-l1-1-0.dll
 0000:fffd9000       .debug$S                   0000000180000000     ucrt:api-ms-win-crt-runtime-l1-1-0.dll
 0000:fffd9000       .debug$S                   0000000180000000     ucrt:api-ms-win-crt-stdio-l1-1-0.dll
 0000:fffd9000       .debug$S                   0000000180000000     ucrt:api-ms-win-crt-stdio-l1-1-0.dll
 0000:fffd9000       .debug$S                   0000000180000000     ucrt:api-ms-win-crt-stdio-l1-1-0.dll
 0000:fffd9000       .debug$S                   0000000180000000     ucrt:api-ms-win-crt-stdio-l1-1-0.dll
 0000:fffd9000       .debug$S                   0000000180000000     ucrt:api-ms-win-crt-stdio-l1-1-0.dll
 0000:fffd9000       .debug$S                   0000000180000000     ucrt:api-ms-win-crt-stdio-l1-1-0.dll
 0000:fffd9000       .debug$S                   0000000180000000     ucrt:api-ms-win-crt-stdio-l1-1-0.dll
 0000:fffd9000       .debug$S                   0000000180000000     ucrt:api-ms-win-crt-stdio-l1-1-0.dll
 0000:fffd9000       .debug$S                   0000000180000000     ucrt:api-ms-win-crt-stdio-l1-1-0.dll
 0000:fffd9000       .debug$S                   0000000180000000     ucrt:api-ms-win-crt-stdio-l1-1-0.dll
 0000:fffd9000       .debug$S                   0000000180000000     ucrt:api-ms-win-crt-string-l1-1-0.dll
 0000:fffd9000       .debug$S                   0000000180000000     ucrt:api-ms-win-crt-string-l1-1-0.dll
 0000:fffd9000       .debug$S                   0000000180000000     ucrt:api-ms-win-crt-string-l1-1-0.dll
 0000:fffd9000       .debug$S                   0000000180000000     ucrt:api-ms-win-crt-string-l1-1-0.dll
 0000:fffd9000       .debug$S                   0000000180000000     ucrt:api-ms-win-crt-string-l1-1-0.dll
 0000:fffd9000       .debug$S                   0000000180000000     ucrt:api-ms-win-crt-string-l1-1-0.dll
 0000:fffd9000       .debug$S                   0000000180000000     ucrt:api-ms-win-crt-string-l1-1-0.dll
 0000:fffd9000       .debug$S                   0000000180000000     ucrt:api-ms-win-crt-string-l1-1-0.dll
 0000:fffd9000       .debug$S                   0000000180000000     kernel32:KERNEL32.dll
 0000:fffd9000       .debug$S                   0000000180000000     kernel32:KERNEL32.dll
 0000:fffd9000       .debug$S                   0000000180000000     kernel32:KERNEL32.dll
 0000:fffd9000       .debug$S                   0000000180000000     kernel32:KERNEL32.dll
 0000:fffd9000       .debug$S                   0000000180000000     kernel32:KERNEL32.dll
 0000:fffd9000       .debug$S                   0000000180000000     kernel32:KERNEL32.dll
 0000:fffd9000       .debug$S                   0000000180000000     kernel32:KERNEL32.dll
 0000:fffd9000       .debug$S                   0000000180000000     kernel32:KERNEL32.dll
 0000:fffd9000       .debug$S                   0000000180000000     kernel32:KERNEL32.dll
 0000:fffd9000       .debug$S                   0000000180000000     kernel32:KERNEL32.dll
 0000:fffd9000       .debug$S                   0000000180000000     kernel32:KERNEL32.dll
 0000:fffd9000       .debug$S                   0000000180000000     kernel32:KERNEL32.dll
 0000:fffd9000       .debug$S                   0000000180000000     kernel32:KERNEL32.dll
 0000:fffd9000       .debug$S                   0000000180000000     kernel32:KERNEL32.dll
 0000:fffd9000       .debug$S                   0000000180000000     kernel32:KERNEL32.dll
 0000:fffd9000       .debug$S                   0000000180000000     kernel32:KERNEL32.dll
 0000:fffd9000       .debug$S                   0000000180000000     kernel32:KERNEL32.dll
 0000:fffd9000       .debug$S                   0000000180000000     kernel32:KERNEL32.dll
 0000:fffd9000       .debug$S                   0000000180000000     kernel32:KERNEL32.dll
 0000:fffd9000       .debug$S                   0000000180000000     kernel32:KERNEL32.dll
 0000:fffd9000       .debug$S                   0000000180000000     kernel32:KERNEL32.dll
 0000:fffd9000       .debug$S                   0000000180000000     kernel32:KERNEL32.dll
 0000:fffd9000       .debug$S                   0000000180000000     kernel32:KERNEL32.dll
 0000:fffd9000       .debug$S                   0000000180000000     kernel32:KERNEL32.dll
 0000:fffd9000       .debug$S                   0000000180000000     kernel32:KERNEL32.dll
 0000:fffd9000       .debug$S                   0000000180000000     kernel32:KERNEL32.dll
 0000:fffd9000       .debug$S                   0000000180000000     kernel32:KERNEL32.dll
 0000:fffd9000       .debug$S                   0000000180000000     kernel32:KERNEL32.dll
 0001:0000134c       addRefToVerify             000000018000234c f   libobjfree002.obj
 0001:000013c0       agentThreadWrapper         00000001800023c0 f   libobjfree002.obj
 0001:00001514       check_option               0000000180002514 f   libobjfree002.obj
 0001:000016d8       envStorageFunc             00000001800026d8 f   libobjfree002.obj
 0001:00001928       file_basename              0000000180002928 f   libobjfree002.obj
 0001:000022fc       rawMonitorFunc             00000001800032fc f   libobjfree002.obj
 0001:000027b4       startAgentThreadWrapper    00000001800037b4 f   libobjfree002.obj
 0001:00002ae0       syncDebuggeeStatus         0000000180003ae0 f   libobjfree002.obj
 0001:00002d68       capture_previous_context   0000000180003d68 f   MSVCRT:gs_report.obj
 0001:00002ddc       ?__scrt_initialize_thread_safe_statics@@YAHXZ 0000000180003ddc f   MSVCRT:thread_safe_statics.obj
 0001:00002eac       ?__scrt_uninitialize_thread_safe_statics@@YAXXZ 0000000180003eac f   MSVCRT:thread_safe_statics.obj
 0001:00002f50       $$000000                   0000000180003f50     MSVCRT:amdsecgs.obj
 0001:00002f80       ?dllmain_crt_dispatch@@YAHQEAUHINSTANCE__@@KQEAX@Z 0000000180003f80 f   MSVCRT:dll_dllmain.obj
 0001:00002fd0       ?dllmain_crt_process_attach@@YAHQEAUHINSTANCE__@@QEAX@Z 0000000180003fd0 f   MSVCRT:dll_dllmain.obj
 0001:000030e8       ?dllmain_crt_process_detach@@YAH_N@Z 00000001800040e8 f   MSVCRT:dll_dllmain.obj
 0001:0000316c       ?dllmain_dispatch@@YAHQEAUHINSTANCE__@@KQEAX@Z 000000018000416c f   MSVCRT:dll_dllmain.obj
 0001:00003b80       $$000000                   0000000180004b80     MSVCRT:guard_dispatch.obj
 0001:00003ba0       $$000000                   0000000180004ba0     MSVCRT:guard_xfg_dispatch.obj
 0001:00003bb6       ?fin$0@?0??dllmain_crt_process_attach@@YAHQEAUHINSTANCE__@@QEAX@Z@4HA 0000000180004bb6 f   MSVCRT:dll_dllmain.obj
 0001:00003bcd       ?fin$0@?0??dllmain_crt_process_detach@@YAH_N@Z@4HA 0000000180004bcd f   MSVCRT:dll_dllmain.obj
 0001:00003be6       ?fin$1@?0??dllmain_crt_process_detach@@YAH_N@Z@4HA 0000000180004be6 f   MSVCRT:dll_dllmain.obj
 0001:00003bfa       ?filt$0@?0??dllmain_dispatch@@YAHQEAUHINSTANCE__@@KQEAX@Z@4HA 0000000180004bfa f   MSVCRT:dll_dllmain.obj
 0001:00003c30       __scrt_is_nonwritable_in_current_image$filt$0 0000000180004c30 f   MSVCRT:utility.obj
 0002:00000218       ?__scrt_initialize_tss_var@@3P6AHXZEA 0000000180005218     MSVCRT:thread_safe_statics.obj
 0002:00000340       ?opcLengths@@3QBEB         0000000180005340     libobjfree002.obj
 0002:00002960       GS_ExceptionPointers       0000000180007960     MSVCRT:gs_report.obj
 0002:00003070       $unwind$fprintf            0000000180008070     libobjfree002.obj
 0002:0000307c       $unwind$printf             000000018000807c     libobjfree002.obj
 0002:00003088       $unwind$?NewObject@JNIEnv_@@QEAAPEAV_jobject@@PEAV_jclass@@PEAU_jmethodID@@ZZ 0000000180008088     libobjfree002.obj
 0002:00003088       $unwind$nsk_lcomplain      0000000180008088     libobjfree002.obj
 0002:00003088       $unwind$nsk_ldisplay       0000000180008088     libobjfree002.obj
 0002:00003090       $unwind$nsk_lvdisplay      0000000180008090     libobjfree002.obj
 0002:00003090       $unwind$_RTC_Initialize    0000000180008090     MSVCRT:initsect.obj
 0002:00003090       $unwind$_RTC_Terminate     0000000180008090     MSVCRT:initsect.obj
 0002:00003090       $unwind$?__scrt_initialize_thread_safe_statics@@YAHXZ 0000000180008090     MSVCRT:thread_safe_statics.obj
 0002:0000309c       $unwind$nsk_complain       000000018000809c     libobjfree002.obj
 0002:0000309c       $unwind$nsk_printf         000000018000809c     libobjfree002.obj
 0002:000030a4       $unwind$nsk_lvcomplain     00000001800080a4     libobjfree002.obj
 0002:000030bc       $unwind$nsk_ltrace         00000001800080bc     libobjfree002.obj
 0002:000030bc       $unwind$__report_gsfailure 00000001800080bc     MSVCRT:gs_report.obj
 0002:000030c4       $unwind$nsk_lvtrace        00000001800080c4     libobjfree002.obj
 0002:000030c4       $unwind$__raise_securityfailure 00000001800080c4     MSVCRT:gs_report.obj
 0002:000030c4       $unwind$__scrt_initialize_crt 00000001800080c4     MSVCRT:utility.obj
 0002:000030c4       $unwind$__scrt_initialize_onexit_tables 00000001800080c4     MSVCRT:utility.obj
 0002:000030c4       $unwind$__scrt_release_startup_lock 00000001800080c4     MSVCRT:utility.obj
 0002:000030c4       $unwind$__scrt_uninitialize_crt 00000001800080c4     MSVCRT:utility.obj
 0002:000030c4       $unwind$_onexit            00000001800080c4     MSVCRT:utility.obj
 0002:000030cc       $unwind$nsk_lverify        00000001800080cc     libobjfree002.obj
 0002:000030dc       $unwind$nsk_vprintf        00000001800080dc     libobjfree002.obj
 0002:000030ec       $unwind$?nsk_jni_lverify@@YAHHPEAUJNIEnv_@@HQEBDH1ZZ 00000001800080ec     libobjfree002.obj
 0002:00003100       $unwind$?nsk_jni_check_exception@@YAHPEAUJNIEnv_@@QEBDH@Z 0000000180008100     libobjfree002.obj
 0002:0000311c       $unwind$nsk_jvmti_parseOptions 000000018000811c     libobjfree002.obj
 0002:00003138       $unwind$nsk_jvmti_createJVMTIEnv 0000000180008138     libobjfree002.obj
 0002:0000314c       $unwind$Java_nsk_jvmti_unit_FollowReferences_FollowRefObjects_resetTags 000000018000814c     libobjfree002.obj
 0002:0000314c       $unwind$VMDeath            000000018000814c     libobjfree002.obj
 0002:0000314c       $unwind$addRefToVerify     000000018000814c     libobjfree002.obj
 0002:0000314c       $unwind$nsk_jvmti_resetAgentData 000000018000814c     libobjfree002.obj
 0002:0000314c       $unwind$__scrt_initialize_default_local_stdio_options 000000018000814c     MSVCRT:default_local_stdio_options.obj
 0002:0000314c       $unwind$?dllmain_crt_dispatch@@YAHQEAUHINSTANCE__@@KQEAX@Z 000000018000814c     MSVCRT:dll_dllmain.obj
 0002:0000314c       $unwind$DllMain            000000018000814c     MSVCRT:dll_dllmain_stub.obj
 0002:0000314c       $unwind$__GSHandlerCheck   000000018000814c     MSVCRT:gshandler.obj
 0002:0000314c       $unwind$?__scrt_uninitialize_thread_safe_statics@@YAXXZ 000000018000814c     MSVCRT:thread_safe_statics.obj
 0002:0000314c       $unwind$__scrt_acquire_startup_lock 000000018000814c     MSVCRT:utility.obj
 0002:0000314c       $unwind$__scrt_dllmain_after_initialize_c 000000018000814c     MSVCRT:utility.obj
 0002:0000314c       $unwind$__scrt_dllmain_before_initialize_c 000000018000814c     MSVCRT:utility.obj
 0002:0000314c       $unwind$__scrt_dllmain_crt_thread_attach 000000018000814c     MSVCRT:utility.obj
 0002:0000314c       $unwind$__scrt_dllmain_crt_thread_detach 000000018000814c     MSVCRT:utility.obj
 0002:0000314c       $unwind$__scrt_dllmain_uninitialize_c 000000018000814c     MSVCRT:utility.obj
 0002:0000314c       $unwind$__scrt_dllmain_uninitialize_critical 000000018000814c     MSVCRT:utility.obj
 0002:0000314c       $unwind$atexit             000000018000814c     MSVCRT:utility.obj
 0002:00003154       $unwind$nsk_jvmti_lverify  0000000180008154     libobjfree002.obj
 0002:00003168       $unwind$exitOnError        0000000180008168     libobjfree002.obj
 0002:00003178       $unwind$check_option       0000000180008178     libobjfree002.obj
 0002:00003178       $unwind$_DllMainCRTStartup 0000000180008178     MSVCRT:dll_dllmain.obj
 0002:00003188       $unwind$Java_nsk_share_jvmti_ArgumentHandler_getAgentOptionsString 0000000180008188     libobjfree002.obj
 0002:0000319c       $unwind$Java_nsk_jvmti_unit_FollowReferences_FollowRefObjects_getTag 000000018000819c     libobjfree002.obj
 0002:0000319c       $unwind$Java_nsk_share_jvmti_DebugeeClass_checkStatus 000000018000819c     libobjfree002.obj
 0002:0000319c       $unwind$agentThreadWrapper 000000018000819c     libobjfree002.obj
 0002:000031ac       $unwind$Agent_Initialize   00000001800081ac     libobjfree002.obj
 0002:000031ac       $unwind$startAgentThreadWrapper 00000001800081ac     libobjfree002.obj
 0002:000031c8       $unwind$syncDebuggeeStatus 00000001800081c8     libobjfree002.obj
 0002:000031c8       $unwind$__scrt_dllmain_exception_filter 00000001800081c8     MSVCRT:utility.obj
 0002:000031dc       $unwind$Java_nsk_share_jvmti_DebugeeClass_resetAgentData 00000001800081dc     libobjfree002.obj
 0002:000031e4       $unwind$MA_checkStatus     00000001800081e4     libobjfree002.obj
 0002:000031f8       $unwind$Java_nsk_jvmti_unit_FollowReferences_FollowRefObjects_setTag 00000001800081f8     libobjfree002.obj
 0002:00003210       $unwind$Java_nsk_jvmti_unit_FollowReferences_FollowRefObjects_addRefToVerify 0000000180008210     libobjfree002.obj
 0002:0000322c       $unwind$rawMonitorFunc     000000018000822c     libobjfree002.obj
 0002:00003244       $unwind$envStorageFunc     0000000180008244     libobjfree002.obj
 0002:0000325c       $unwind$ObjectFree         000000018000825c     libobjfree002.obj
 0002:00003274       $unwind$Java_nsk_jvmti_ObjectFree_objfree002_setTag 0000000180008274     libobjfree002.obj
 0002:00003288       $unwind$capture_previous_context 0000000180008288     MSVCRT:gs_report.obj
 0002:00003294       $unwind$__GSHandlerCheckCommon 0000000180008294     MSVCRT:gshandler.obj
 0002:000032a0       $xdatasym                  00000001800082a0     MSVCRT:amdsecgs.obj
 0002:000032a4       $unwind$?dllmain_crt_process_attach@@YAHQEAUHINSTANCE__@@QEAX@Z 00000001800082a4     MSVCRT:dll_dllmain.obj
 0002:000032e0       $unwind$?fin$0@?0??dllmain_crt_process_attach@@YAHQEAUHINSTANCE__@@QEAX@Z@4HA 00000001800082e0     MSVCRT:dll_dllmain.obj
 0002:000032e0       $unwind$?fin$0@?0??dllmain_crt_process_detach@@YAH_N@Z@4HA 00000001800082e0     MSVCRT:dll_dllmain.obj
 0002:000032e0       $unwind$?fin$1@?0??dllmain_crt_process_detach@@YAH_N@Z@4HA 00000001800082e0     MSVCRT:dll_dllmain.obj
 0002:000032e8       $unwind$?dllmain_crt_process_detach@@YAH_N@Z 00000001800082e8     MSVCRT:dll_dllmain.obj
 0002:0000333c       $unwind$?dllmain_dispatch@@YAHQEAUHINSTANCE__@@KQEAX@Z 000000018000833c     MSVCRT:dll_dllmain.obj
 0002:00003364       $unwind$?filt$0@?0??dllmain_dispatch@@YAHQEAUHINSTANCE__@@KQEAX@Z@4HA 0000000180008364     MSVCRT:dll_dllmain.obj
 0002:0000336c       $unwind$__scrt_is_nonwritable_in_current_image 000000018000836c     MSVCRT:utility.obj
 0002:0000338c       $unwind$__scrt_is_nonwritable_in_current_image$filt$0 000000018000838c     MSVCRT:utility.obj
 0002:00003394       $unwind$__scrt_fastfail    0000000180008394     MSVCRT:utility_desktop.obj
 0002:000033a4       $unwind$__security_init_cookie 00000001800083a4     MSVCRT:gs_support.obj
 0002:000033b0       $unwind$__isa_available_init 00000001800083b0     MSVCRT:cpu_disp.obj
 0002:000033c0       $xdatasym                  00000001800083c0     MSVCRT:guard_dispatch.obj
 0002:000033c8       $xdatasym                  00000001800083c8     MSVCRT:guard_xfg_dispatch.obj
 0002:000033d0       .edata                     00000001800083d0     objfree002.exp
 0002:000033f8       rgpv                       00000001800083f8     objfree002.exp
 0002:00003438       rgszName                   0000000180008438     objfree002.exp
 0002:00003478       rgwOrd                     0000000180008478     objfree002.exp
 0002:00003498       szName                     0000000180008498     objfree002.exp
 0002:000034a7       $N00001                    00000001800084a7     objfree002.exp
 0002:000034b6       $N00002                    00000001800084b6     objfree002.exp
 0002:000034c3       $N00003                    00000001800084c3     objfree002.exp
 0002:000034ee       $N00004                    00000001800084ee     objfree002.exp
 0002:0000351a       $N00005                    000000018000851a     objfree002.exp
 0002:0000355f       $N00006                    000000018000855f     objfree002.exp
 0002:0000359c       $N00007                    000000018000859c     objfree002.exp
 0002:000035e4       $N00008                    00000001800085e4     objfree002.exp
 0002:00003624       $N00009                    0000000180008624     objfree002.exp
 0002:00003661       $N00010                    0000000180008661     objfree002.exp
 0002:0000369c       $N00011                    000000018000869c     objfree002.exp
 0002:000036ca       $N00012                    00000001800086ca     objfree002.exp
 0002:000036fb       $N00013                    00000001800086fb     objfree002.exp
 0002:0000372a       $N00014                    000000018000872a     objfree002.exp
 0002:00003759       $N00015                    0000000180008759     objfree002.exp
 0002:0000378e       $N00016                    000000018000878e     objfree002.exp
 0002:00003bf2       .idata$6                   0000000180008bf2     kernel32:KERNEL32.dll
 0002:00003c56       .idata$6                   0000000180008c56     vcruntime:VCRUNTIME140.dll
 0002:00003de8       .idata$6                   0000000180008de8     ucrt:api-ms-win-crt-heap-l1-1-0.dll
 0002:00003e08       .idata$6                   0000000180008e08     ucrt:api-ms-win-crt-runtime-l1-1-0.dll
 0002:00003e2a       .idata$6                   0000000180008e2a     ucrt:api-ms-win-crt-convert-l1-1-0.dll
 0002:00003e4c       .idata$6                   0000000180008e4c     ucrt:api-ms-win-crt-stdio-l1-1-0.dll
 0002:00003e6c       .idata$6                   0000000180008e6c     ucrt:api-ms-win-crt-string-l1-1-0.dll
 0003:00000000       ?codeAttributeName@@3PEBDEB 0000000180009000     libobjfree002.obj
 0003:00000008       ?lineNumberAttributeName@@3PEBDEB 0000000180009008     libobjfree002.obj
 0003:00000010       ?localVarAttributeName@@3PEBDEB 0000000180009010     libobjfree002.obj
 0003:00000018       ?localVarTypeAttributeName@@3PEBDEB 0000000180009018     libobjfree002.obj
 0003:00000020       ?stackMapAttributeName@@3PEBDEB 0000000180009020     libobjfree002.obj
 0003:00000028       ?callBytes@@3PAEA          0000000180009028     libobjfree002.obj
 0003:0000002c       ?allocBytes@@3PAEA         000000018000902c     libobjfree002.obj
 0003:0001aae0       nsk_context                0000000180023ae0     libobjfree002.obj
 0003:0001aaec       redefineAttempted          0000000180023aec     libobjfree002.obj
 0003:0001aaf0       redefineSucceed            0000000180023af0     libobjfree002.obj
 0003:0001aaf4       agentFailed                0000000180023af4     libobjfree002.obj
 0003:0001aaf8       agentThread                0000000180023af8     libobjfree002.obj
 0003:0001ab00       context                    0000000180023b00     libobjfree002.obj
 0003:0001abb8       agentThreadProc            0000000180023bb8     libobjfree002.obj
 0003:0001abc0       agentThreadArg             0000000180023bc0     libobjfree002.obj
 0003:0001abc8       agent_data                 0000000180023bc8     libobjfree002.obj
 0003:0001abd8       jvmti_env                  0000000180023bd8     libobjfree002.obj
 0003:0001abe0       jvm                        0000000180023be0     libobjfree002.obj
 0003:0001abe8       jni_env                    0000000180023be8     libobjfree002.obj
 0003:0001abf0       currentAgentStatus         0000000180023bf0     libobjfree002.obj
 0003:0001abf4       ?codeAttributeIndex@@3GA   0000000180023bf4     libobjfree002.obj
 0003:0001abf8       checkStatus_func           0000000180023bf8     libobjfree002.obj
 0003:0001ac00       ?lineNumberAttributeIndex@@3GA 0000000180023c00     libobjfree002.obj
 0003:0001ac04       ?localVarAttributeIndex@@3GA 0000000180023c04     libobjfree002.obj
 0003:0001ac08       ?localVarTypeAttributeIndex@@3GA 0000000180023c08     libobjfree002.obj
 0003:0001ac0c       ?stackMapAttributeIndex@@3GA 0000000180023c0c     libobjfree002.obj
 0003:0001ac10       ?stackFrameOffset@@3GA     0000000180023c10     libobjfree002.obj
 0003:0001ac14       ?mode@@3HA                 0000000180023c14     libobjfree002.obj
 0003:0001ac18       ?orig@@3PEBEEB             0000000180023c18     libobjfree002.obj
 0003:0001ac20       ?gen@@3PEAEEA              0000000180023c20     libobjfree002.obj
 0003:0001ac28       ?inputPos@@3PEAEEA         0000000180023c28     libobjfree002.obj
 0003:0001ac30       ?endPos@@3PEBEEB           0000000180023c30     libobjfree002.obj
 0003:0001ac38       ?genPos@@3PEAEEA           0000000180023c38     libobjfree002.obj
 0003:0001ac40       ?markPos@@3PEAEEA          0000000180023c40     libobjfree002.obj
 0003:0001ac48       ?constantPool@@3PEAPEADEA  0000000180023c48     libobjfree002.obj
 0003:0001ac50       ?constantPoolSize@@3GA     0000000180023c50     libobjfree002.obj
 0003:0001ac54       ?constantPoolCount@@3GA    0000000180023c54     libobjfree002.obj
 0003:0001ac58       ?zeroBytes@@3PAEA          0000000180023c58     libobjfree002.obj
 0003:0001ac5c       ?codeLength@@3IA           0000000180023c5c     libobjfree002.obj
 0003:0001ac60       ?map@@3PEAIEA              0000000180023c60     libobjfree002.obj
 0003:0001ac68       ?widening@@3PEACEA         0000000180023c68     libobjfree002.obj
 0003:0001ac70       jvmti                      0000000180023c70     libobjfree002.obj
 0003:0001ac78       result                     0000000180023c78     libobjfree002.obj
 0003:0001ac80       callbacks                  0000000180023c80     libobjfree002.obj
 0003:0001adb8       caps                       0000000180023db8     libobjfree002.obj
 0003:0001adc8       objfree                    0000000180023dc8     libobjfree002.obj
 0003:0001add0       stor                       0000000180023dd0     libobjfree002.obj
 0003:0001b1e0       GS_ExceptionRecord         00000001800241e0     MSVCRT:gs_report.obj
 0003:0001b280       GS_ContextRecord           0000000180024280     MSVCRT:gs_report.obj
 0003:0001b750       ?g_tss_cv@@3U_RTL_CONDITION_VARIABLE@@A 0000000180024750     MSVCRT:thread_safe_statics.obj
 0003:0001b758       ?g_tss_event@@3PEAXEA      0000000180024758     MSVCRT:thread_safe_statics.obj
 0003:0001b760       ?g_tss_mutex@@3U_RTL_CRITICAL_SECTION@@A 0000000180024760     MSVCRT:thread_safe_statics.obj
 0003:0001b788       ?g_sleep_condition_variable_cs@@3P6AHPEAU_RTL_CONDITION_VARIABLE@@PEAU_RTL_CRITICAL_SECTION@@K@ZEA 0000000180024788     MSVCRT:thread_safe_statics.obj
 0003:0001b790       ?g_wake_all_condition_variable@@3P6AXPEAU_RTL_CONDITION_VARIABLE@@@ZEA 0000000180024790     MSVCRT:thread_safe_statics.obj
 0003:0001b79c       ?__proc_attached@@3HA      000000018002479c     MSVCRT:dll_dllmain.obj
 0003:0001b7b0       ?is_initialized_as_dll@@3_NA 00000001800247b0     MSVCRT:utility.obj
 0003:0001b7b1       ?module_local_atexit_table_initialized@@3_NA 00000001800247b1     MSVCRT:utility.obj
 0003:0001b7b8       ?module_local_atexit_table@@3U_onexit_table_t@@A 00000001800247b8     MSVCRT:utility.obj
 0003:0001b7d0       ?module_local_at_quick_exit_table@@3U_onexit_table_t@@A 00000001800247d0     MSVCRT:utility.obj
